:020000041100E9
:10300000002373B52B4D2C4C28006361022601F080
:1030100071F94021FE2221742800284B009601F00E
:10302000BBF9002836D1217CFF222800244B0096D2
:1030300001F0B2F900282DD1224BA2899A4226D163
:10304000E389214A93420DD1204B6361204B2268D2
:10305000002A03D1002B01D043CB43C4280001F048
:1030600087F973BD1B4A934201D00023EFE71A4B47
:103070001A4A1B68934206D9C02304222800217CE7
:103080009B0001F0FFF9114B6361154BDFE7002353
:103090002374EAE7CC233821AC2228009B01217459
:1030A00001F0F0F90028F2D10E4B63610E4BE38181
:1030B0000E4BCCE7F441FF1FA061FF1FAC61FF1F67
:1030C000AE61FF1F59590000830500002141001126
:1030D00060BD001182150000C461FF1F871300004E
:1030E0006CBD0011D9410011AAAAFFFF54BD001107
:1030F000F7B5164B0192C318021D002000938823D8
:103100005B05D3181B685C1C1AD09CB2402C18D8E5
:103110008D781E0CAC466746CD782D023D43AE42FD
:1031200006D1019800280ED110000C70240A4C70B2
:1031300003249BB20733A343D218009B9A42DED3E9
:10314000FEBD4432F9E71000FAE7C046FC0F00006C
:10315000802213B503000324019189B25201073183
:103160009B18A14304305A1A88235B05C3181B68B7
:10317000591C03D190429241104016BD99B240298A
:1031800007D80B000733A343C0189042ECD30020AC
:10319000F3E74430F9E7134B134A1B68126810B584
:1031A000FA24934201D81A00F824104BE4021B6859
:1031B0009A4210D813000E4A12689A420ED3013375
:1031C00007D1F823DB029C4203D10A49054808F0E5
:1031D0003BFD200010BDFC24E402ECE7FE24E402E9
:1031E000F7E7C04600C0071100D0071100E0071143
:1031F00000F00711FFFFFF7FF0B59BB015000490B2
:103200000391402A00D9A0E006AB59801A80FFF74D
:10321000C2FF0400042816D9002206A9FFF768FFA0
:10322000052810D906AB1B88AB420CD1002D07D066
:10323000514B2A000499C01808F006FC002802D15E
:1032400001201BB0F0BD06AB1D8020000699FFF7E2
:103250007FFF041E7BD1069B0793FFF79CFF802313
:103260005B01C618802307001B039E4201D3F8268A
:10327000F60288235B05F31801931B68013302D023
:10328000019808F0E9FA3D49019808F0DDFC3B1D82
:103290000293331D05938822029B52059B181B68DD
:1032A00008935A1C3CD044219AB20091402A04D879
:1032B0000320D11D814389B2009103991B0C8B42DD
:1032C00024D0402A22D80122300008A9FFF710FF9D
:1032D000021E1BD1380008A9FFF70AFF04000428CA
:1032E00031D9009A059B9B1880225201B218934253
:1032F00040D288235B05C118009A09A808F004FC95
:103300001D4B009A09A9F01808F07EFC009A029B58
:103310009446634402931A4B029AFB189A42BAD31A
:1033200088235B05FC1821680198013908F08CFCA2
:10333000200008F091FA039A07AB5A8030000799F1
:10334000FFF706FF0400002C03D1002079E70428D2
:10335000FBD988235B05E018069908F075FC032368
:10336000EA1C9A4300D16BE7034B0499E01808F07C
:103370004BFC65E70424ECE704000011FFFFFF7F2E
:10338000F80F0000F7B505001400402A21D80027E7
:1033900001AE71803780FFF7FEFE042816D93A008F
:1033A0003100FFF7A5FE042810D93688BC420BD0A7
:1033B000BD4209D0221CB44200D9321C064B92B245
:1033C000C118280008F0A0FB30B2FEBDC04300B217
:1033D000FBE703204042F8E70400001137B5042260
:1033E00004000D0001A81649FFF7CCFF02000428D5
:1033F0000BD1019BA34208D3AB4204D0104901A8D2
:103400000195FFF7F9FE01203EBD0E4C2368200018
:10341000019308F021FA019920000139019108F087
:1034200013FC80235B01E418074B9C42EED104227D
:10343000034901A80195FFF7DFFE0020E4E7C0463D
:103440005555000000C007110000081130B589B0C3
:1034500008F03AFA10226946254808F06DF9254B24
:10346000009A9A420ED1019B029A0F2B33D8002169
:1034700001240698013B08D2002900D00292029B49
:10348000013331D10023029325E0551CF2D1020013
:103490002100EFE710341022200004A908F04CF9B5
:1034A000029B013301D1069B0293882304995B059B
:1034B000C918059B06981A03120B049105928142C4
:1034C00003D02B4201D108F01FFB019B013B01936C
:1034D000019B002BDED1029B002B03D004930498A8
:1034E0004168084709B030BDE025014C2D03EFE7E6
:1034F00000000111504859368022F8B5964C974B80
:10350000D200002120001C6008F0BEF92300944A7C
:1035100088331A60934B1A786A23002A00D011333B
:10352000E3620A232365904B37221B780820A363AC
:103530008E4B2118E361102323628D4B3B25636181
:10354000C823DB00A36123008C331A602823013ACF
:10355000E26320646364CA67043A211DCA672100DC
:10356000BC310D602100C03108602100C4310B6006
:1035700021000635CC310D602100083DC8310D60B9
:103580002100D0310A602200D43210602200D832EB
:10359000136022000227E032210017604222DC3152
:1035A0000A6021001B3DE4310D602100E831086014
:1035B0002100EC310B6023000521F4331960230056
:1035C000F0331A602300183290331A6023009433CA
:1035D000186023001E3A98331A60AF23DB00236083
:1035E000644BFA262363644B644DE360644BF03113
:1035F000A3642300FF31FC33B600A16021611E608B
:10360000A5627325E5656D3D6565A56596255D4AF1
:10361000AD00E264666258606766A566002709250A
:10362000A767E566584F594D606720002567E26738
:103630003A6015279C30676007001A203860200028
:10364000A0300700212038602000A83007004C4837
:1036500038602000F830066026006427A436376002
:1036600026005F3FAC3637602600033FB036376038
:103670002600C637B436376026000027B8363760D4
:1036800038269E60424E96205E64424E5A66DE6147
:10369000414E9A645E62F53EFF3E9E621E269A6728
:1036A000354A8000DE661F675F67DD651D6618624C
:1036B000DA67BE23394A5B00E250394BD8382350D1
:1036C00004302250C4225200A350C623E4205B00E1
:1036D000E1500433334AE1503349344BD16034492B
:1036E000800019503349E938FF3819503249043005
:1036F000195032493248D16132491163324951631C
:103700001900F4310860CE20304940001160304982
:10371000195019002F48F83108602F49D1658221CE
:103720002E4A89005A501A002D490832D1671A00D2
:103730002C49B432116088212B4A89005A501A0052
:103740002A49883211602A4ADA6408F0F5F8012023
:1037500007F09AFFF8BDC0460004FF1F4464FF1F36
:10376000206FFF1F3444FF1F4A0AFF1F3A07000063
:1037700080C3C9019A020000DC0500006A1800003D
:1037800050C3000088130000F009FF1F204E000006
:103790006509FF1F68100000C409000040420F00C7
:1037A00010270000FC00FF1FC11BFF1F0000FF1FB0
:1037B000152CFF1FA52FFF1F3D2EFF1F811FFF1F71
:1037C0007126FF1F9D1FFF1F4921FF1F0D1FFF1F98
:1037D0009528FF1F7D29FF1FD918FF1FA127FF1F55
:1037E000C524FF1FD124FF1F0D1EFF1FC51EFF1F75
:1037F000851DFF1FF0B502250124604B91B01D709F
:1038000002935F4B5F4E1C705F4F03933368002140
:103810002800FB7006F00EFE280006F005FD0023D0
:10382000984205D0FA78552A02D0332A00D098E081
:103830003360042006F066FF07F0FEFFFFF75CFE32
:1038400007F04AFF1F2201240021504B10AD1A70CF
:103850004F4B1C704F4B19704F4B19689143163AE0
:103860000A431A60602219689143403A0A431A6079
:1038700007F0E2FE07F018FFC120FF21474B800050
:103880001A588A431A50C522920098588843BF3963
:10389000014399509858424908408021C901014389
:1038A000802099509958C0050902090A014399508E
:1038B00080213C48490108F08FF8032322003A494F
:1038C00001940093394808F007F92C22384905A8DB
:1038D00008F01AF905AC61782078023406F0C4FCCF
:1038E000A542F8D1334C344B226803201A40A02360
:1038F000DB0213432360802322689B04134323606D
:1039000022682E4B1A4080239B03134323602C4ACA
:103910002C4B934200D8012007F026FF08F09CF8BA
:1039200080232268DB0413432360029B187808F08D
:1039300023F9039B1878C0B208F046F808F0F4F8B1
:103940002149042008F030F806F0A8FE00F0ACF899
:1039500000F0EEFD00F096FE00F010FA002011B02D
:10396000F0BD00932100184A042007F0DDFF8023FA
:10397000DB059C62FFF76AFD5BE7C0464A0AFF1F52
:103980003444FF1F34F00040D061FF1F480AFF1F7E
:10399000490AFF1F680AFF1FBCF0004000E100E079
:1039A000FF00FFFF3844FF1FBC56FF1F3854FF1FA6
:1039B00078BC001114F00040FF7FF8FFFFFF9FFF6D
:1039C0000080FF1F206FFF1F3B00010870B500251E
:1039D0002549264A26484D6308CA1B051B0DED18CC
:1039E0008242F9D100268022224B92058B63092165
:1039F000214B224C1E62224B1120DA67214BDA68E0
:103A00008A43DA609A6820490A409A60266008F082
:103A100013F9112007F030FF636C1C4A13406364F4
:103A20001B4C1C4A6C43200C0400642390420AD8AF
:103A3000FA223300D200904205D9174B0A21C01850
:103A400007F0BAFEC3B2154A11201372D48007F0F2
:103A500023FF134B1B78002B04D1124B1021187835
:103A600008F002F870BDC046000005408807054018
:103A700000080540FF01000000F000400038004051
:103A800004E100E03CF00040FFDFFFFFFFFDFFFF2F
:103A9000AE060000B70B000030F8FFFFB861FF1F53
:103AA000F263FF1FF061FF1F002210B5110011200B
:103AB00007F0B2FE10BD0000F8B500230925374F0E
:103AC000374C3B62E3681120AB43E36007F0D4FE60
:103AD000112008F0B1F8112007F0CEFD4023226834
:103AE00080261343236080236268DB0213436360F4
:103AF000A3682C4A3343A360A36828001340A36043
:103B00008023A2689B0113431022A360236C02212F
:103B100093432364236C0F3A1343236480235B0194
:103B20003B62226B204B1A402263626B1A40626335
:103B3000A26B1A40A263E26B1340E363E3681B4A83
:103B40001340E36006F090FB2800012106F0A0FC82
:103B50008023174A9B00516C11200B43536407F0DC
:103B600013FEFD21134B144A89005A508023C720AD
:103B7000E26B5B031343E363E36880001D430F4B79
:103B8000E56019580E4A1140802212020A431A5069
:103B9000802292051A600B4B5E63F8BD00F0004076
:103BA0003CF00040FFFFDFFFEFFFEFFFFFFF7FFF75
:103BB000003800400000FF1FCD39001100E100E097
:103BC000FF00FFFF0000054030B503A804880B206C
:103BD000002C0ED14968074D087849780902014345
:103BE0000A20A94205D1012120001980024B1B7A2D
:103BF000137030BD192A0000B861FF1FF7B515001A
:103C000008AA16884A680F4F147852781202224385
:103C10000A24BA4214D10122DBB2019200962A0092
:103C200007F08CFC041E0BD1074B1B68002B07D040
:103C300068782A7800021043424250410130984788
:103C40002000FEBD022900003C61FF1F30B50125A8
:103C500003790400BFB02B4211D00A49408806F016
:103C6000D9FF28420BD0084B01A95B8D4D800B80FA
:103C7000064B00221B7A60880B7104F0BDF83FB040
:103C800030BDC0463461FF1F6840FF1FB861FF1F91
:103C900010B50549054806F073FF0421044A05489C
:103CA00006F030FF10BDC0463461FF1FFFFF00006B
:103CB000A4BC00116840FF1F10B5024804F01EFFAD
:103CC00010BDC0464D3C0011062310B58370103363
:103CD0000371443B43712A3383714433C37100231E
:103CE0000222012103720E4B027041701C88817206
:103CF0004472197A0273C1729A784273DA788273C5
:103D00000322C2731A7902745A7942740C228274A3
:103D10009A79C274DB7903751123C370152010BD25
:103D2000B861FF1F10B5142007F026FE124B1422B5
:103D30000021186007F0A8FD002007F00DFE01200B
:103D400007F002FE022007F0D7FD032004F07AF905
:103D5000042006F08FF9052003F0B8FB062004F0DC
:103D600085F8072001F04EFA082006F0ABFE092086
:103D700001F036F810BDC0464061FF1F07F03CFE61
:103D8000012007F031FD07F09FFE0000094B10B540
:103D90000400984205D0012904D12000064906F00C
:103DA000EFFE10BD0229FCD1013904F065FE0028A8
:103DB000F3D0F6E7FEFF00006661FF1F70B50D7AD5
:103DC000100004AA2C00168810221440154220D19D
:103DD000002E20D10A78022A18D14A685178157825
:103DE0000E4A09022943914205D00D4A914209D059
:103DF0001C800A2404E014220A491A8007F084FE79
:103E0000200070BD0C2208491A80F7E71C800124AD
:103E1000F6E70824F4E70B24F2E7C046F3FF0000BE
:103E2000F4FF0000C042FF1F84BD001110B5040064
:103E30000749084806F0A4FE074804F09FFD00204B
:103E4000E40704D50721054A054806F05BFE10BDCE
:103E50006661FF1FFFFF00008D3D0011E8BC0011EF
:103E6000AC40FF1F00B50C4BBFB01A780B4902A83D
:103E700000F0C2FC6B4680B2D880002809D06A46A8
:103E8000074B01A91B889380064B0022188803F07A
:103E9000B3FF3FB000BDC0464461FF1F4561FF1F37
:103EA0000641FF1F1042FF1F00B50C4BBFB01A7830
:103EB0000B4902A801F0E6FE6B4680B2D8800028CC
:103EC00009D06A46074B01A95B8D9380064B0022FF
:103ED000188803F091FF3FB000BDC0466E61FF1F20
:103EE0006F61FF1FAC40FF1F1042FF1FF7B50E00B0
:103EF000377A1C0008AB11003D001A8820231D40B2
:103F00001F423CD13378022B3BD173681F785B781A
:103F10001B023B431E4FBB4208D01E4FBB4214D076
:103F20001D4DAB4221D00A252800FEBD002A2AD112
:103F3000142C2AD82200F06807F0E6FD174B1C70FD
:103F4000012CF1D9FFF7B0FFEEE7002A1BD1202C9E
:103F50001BD82200F06807F0D7FD114B04211C701C
:103F6000104B187807F080FDDEE7E3B201240092E1
:103F700001940A00310007F0E1FA0500D4E70825B2
:103F8000D2E70125D0E70B25CEE70D25CCE7C046CB
:103F9000F3FF0000F4FF0000022900006E61FF1F24
:103FA0004461FF1FF061FF1F332310B5040003704D
:103FB0000A220749013007F0A7FD064B0F201B68B6
:103FC0001A0AE37222731A0C1B0E6273A37310BDDC
:103FD000B861FF1FE061FF1F30B5012503790400C0
:103FE000BFB02B4213D00B49408806F013FE284285
:103FF0000DD06A46084B02A81B889380FFF7D4FFB8
:104000006B46D8800022608801A903F0F5FE3FB01E
:1040100030BDC0466661FF1F0641FF1F10B5024854
:1040200004F06CFD10BDC046D93F001170B51600FC
:1040300004AA148805AA15784A68507811780002F5
:104040002A4A0843801805284BD807F0F5FC0313CB
:104050001E29343F0720042C0BD80522121BAA422C
:1040600000D92A0022491A803000091907F04CFDB6
:10407000002070BD0720112CFBD81222121BAA426F
:1040800000D92A001B491A80EEE707200E2CF0D831
:104090000F22121BAA4200D92A0017491A80E3E70F
:1040A0000720032CE5D80422121BAA4200D92A00BB
:1040B00012491A80D8E70720032CDAD80422121BF1
:1040C000AA4200D92A000E491A80CDE70720032C06
:1040D000CFD80422121BAA4200D92A0009491A800B
:1040E000C2E700220A201A80C3E7C046DCD5FFFFE2
:1040F00033BD00118C61FF1F23BD00111EBD0011D7
:1041000019BD001114BD001110B50D21024A03485C
:1041100006F0F8FC10BDC04608BD00111C41FF1F91
:10412000F0B50024274E85B03000B47100F0E2F8FD
:10413000254D264BEA89297C9A422FD10423300051
:1041400003AA00F057F90400300000F011F9012330
:10415000B371002C34D16B4699892B68C9BA4B4393
:1041600029891B4A1B145B1853806B46D9896B68DD
:1041700049BA89B24B4369891B0C5B181548191C55
:104180001BB2834200DD011C0B0400D50021138803
:10419000918001331380200005B0F0BD022722007A
:1041A00003AB3000009700F0F7F80E230400297CE1
:1041B0000122300000976B4400F0EEF80443C3E79F
:1041C0001C00E8E7F441FF1FA061FF1F830500000A
:1041D000B861FF1F0F27000073B5234E300000F0B9
:1041E00089F8224D07236A463000297C00F002F945
:1041F00004003000002C33D16B461B787F2B2FD866
:1042000000F0B6F86B46D878F02302041B031A407E
:104210006B469B8816495BBA9BB21A432B68000910
:1042200053432A891B0C9B184B806B465A789B780A
:1042300012031B011A436B68024353436A891B0C28
:104240009B180C481A1C1BB2834200DD021C13048D
:1042500000D500220B888A8001330B80200076BDB8
:1042600000F086F80124F9E7F441FF1FA061FF1F69
:10427000B861FF1F0F27000070B5114C237C002B85
:104280000FD0382B0ED10F4D280000F033F8CC237F
:10429000AC222800217C9B0100F0F4F8280000F0FB
:1042A00067F870BD084BE2899A42FAD1054D2800A3
:1042B00000F020F800222800217C00F0C5F8EDE78E
:1042C000A061FF1FF441FF1F8305000010B5084BDC
:1042D0001A7C002A09D05B69002B06D09847041E7F
:1042E00001D0FEF78DFE200010BD0124F9E7C04685
:1042F000A061FF1F70B5C17905000C00631E9C41D1
:104300001A4BE402E41849000460C9B2007906F0CF
:10431000F5F8E979687949000131C9B206F0EEF89B
:10432000E8790930C0B207F0A7F90023E3666133EA
:104330002360AA795B3B002A0ED022689A43023B95
:10434000134323600A23E3610733236200232363BB
:10435000A3630133E36370BD22689A4302231343CE
:104360002360462363610633A361EFE700500040FA
:1043700070B5002504000368DD66C0790930C0B25D
:1043800007F07AFA2900207906F054F829006079BC
:1043900006F050F870BD0000F8B51E0006AB1D78A1
:1043A000002304681700E366616007F08DFA0123BB
:1043B0008022E3662B0027615200013B08D207F000
:1043C000BBFB08200A4A1168002D03D12800F8BD64
:1043D0002261F2E7236F034203D02369013D33706A
:1043E000013613685B1A032BEED90125EEE7C046B0
:1043F0006008FF1F70B51C00002305681600EB66FF
:10440000696007F061FA01238022EB662300520005
:10441000013B08D207F090FB08200A4A1168002CE3
:1044200003D1200070BD2A61F2E72B6F034203D055
:104430002B69013C3370013613685B1A032BEED9EC
:104440000124EEE76008FF1F002370B50468150023
:10445000E366616007F038FA0123E366256107F03F
:104460006BFB8020064A80001168636B034205D114
:1044700013685B1A032BF8D9012070BD0020FCE7FC
:104480006008FF1F70B51D00002304681600E36676
:10449000616007F019FA0123E36626610F33626B4E
:1044A0001A42FCD02B0A23611023626B1A42FCD003
:1044B000EDB2256107F040FB8020074A80001168BB
:1044C000636B034205D113685B1A032BF8D90120F3
:1044D00070BD0020FCE7C0466008FF1F70B51E00DD
:1044E000002305681400EB66696007F0EDF901230D
:1044F000A619EB660F33B4420ED107F01DFB8020E6
:104500000A4A800011686B6B03420CD113685B1A76
:10451000032BF8D9012070BD21782961696B1942FC
:10452000FCD00134E7E70020F5E7C0466008FF1F34
:1045300010B5084CE368002B08D18022064B5202CC
:104540001B689B186360054B1B68236007F01CFB0E
:10455000A06010BDE061FF1FC8F00040CCF000403B
:1045600070B5184A936A916A9942FBD116498A68D4
:104570009A421FD39A1A8B60144B0126186893B283
:10458000D202D20E4343424300204C681B0A1B193F
:1045900012029B180E4C0A684B60551CA3420CD8A3
:1045A000002801D04B600A600A4A136008680A4B71
:1045B000186070BD581E821ADDE7084A30009B184B
:1045C0002A00EAE700F00040E061FF1F140AFF1F25
:1045D00040420F00C8F00040CCF00040C0BDF0FFEA
:1045E00070B51F4C23793F2B01D93F2323711D4BFD
:1045F00022791A701878C0B207F0EEFA18231A4917
:104600001A4A0B801A4913800B805380A3791949E9
:1046100080200B800C21938001334B43164D191CD5
:104620000001834200D9011C2980D1806379002BCD
:1046300011D101336371237A012B01D80223237234
:104640006279237A0D4853430A21584307F0B4F89E
:104650000B4D286070BDA02BEDD9A023EAE7C04622
:10466000D461FF1F480AFF1F0E42FF1FE043FF1FD8
:104670000C42FF1F0A42FF1F0842FF1F7102000089
:10468000C461FF1FF8B514210020FEF7A7FE114CEE
:10469000011E114D09D10C22104BC1CBC1C4280001
:1046A00007F0F2F8FFF79CFFF8BD0C2220000C4940
:1046B000FEF768FE0C2802D0084B43CB43C40C2203
:1046C00028000849FEF75EFE0C28EBD00C220021E2
:1046D000E5E7C046D461FF1FA061FF1F78BD001150
:1046E000FC0C0000F50C0000F0B51D4C8022A54428
:1046F0000400882069465201400507F08DFA902297
:1047000012016A441300200032C832C316C816C30F
:104710008023144C144FA6689B033343A3603B6073
:1047200007F0FAF88823A0685B05C01807F094F832
:104730000025882329008022A0685B05C018401945
:104740006944520007F060FA80230135FF355B01B0
:104750009D42EED1A6603E60044B9D44F0BDC04634
:10476000FCEFFFFF5043FF1F9808FF1F04100000DD
:10477000F0B5040087B0002825D0684607F024F87B
:104780001B4C022806D106226946200007F05CF97E
:10479000002816D06946002301250F262F00E25C71
:1047A000013310091030874038002F003240974005
:1047B0003A0002434A610439062BEFD16846FFF7FD
:1047C00093FF07B0F0BD182269460A4807F024FAA3
:1047D0006A46A300D358013305D01822FF2168464A
:1047E00007F052F8EAE70134062CF1D1E9E7C046B8
:1047F0006509FF1F00090011F0B5002504000E0037
:1048000085B0AA4200D186E04B1C087801934B7812
:104810008978377909021943F3783F061B040B4363
:104820001F43039720706570252800D196E033D888
:10483000112813D807F088F96900280128012801F8
:104840002801AA00B800B100280128012801280188
:10485000280128012801280102012201232800D172
:10486000DBE0DB2800D031E1042A00D8ACE01025E1
:10487000052A05D0551F2A003800711D07F044F99C
:1048800005223100200007F03FF92A003900601DA1
:1048900007F03AF905353EE0562859D010D83328AC
:1048A00000D19DE0552839D02628DAD19D4B29002A
:1048B000132218001D0006F0E7FFFEF7A1FB5CE0E5
:1048C000712800D177E0722800D180E0602800D103
:1048D0008BE0DC28C5D1022A00D875E07378BFB21E
:1048E0006370B378A370032A05D0033A390092B2FB
:1048F000F01CFEF781FC10223900E01CFEF742FD9F
:10490000C51C002807DA60705CE00C222000864994
:1049100007F0FAF80C25280005B0F0BD013A834DE8
:104920000C2A13D8002A0AD02800019907F0ECF8C5
:10493000FFF756FE0C2228007D49FEF75DFC29009A
:104940000C22601C07F0E0F80D25E4E70C22EBE7F1
:10495000764D784B2A0043CB43C2E9E7013A714DCB
:104960000C2A11D8002A08D00199280007F0CCF8A9
:104970000C2228007049FEF73FFC29001322601C1E
:1049800007F0C2F81425C6E70C22EDE705226B49B3
:10499000601C07F0B9F80625BDE712226849601CC3
:1049A00007F0B2F81325B6E708226649601C07F045
:1049B000ABF80925AFE77178F02905D8624B188864
:1049C00001F0BCFD0225A6E7FF236370FAE75F4B09
:1049D000012A03D072789A706270F3E79B78F4E74B
:1049E0002000FFF7E1FA050095E7013A574B584DD3
:1049F000082A0DD8002A0DD00121280059700199EC
:104A000007F082F801F072F808222900601CCEE756
:104A10000822F1E700225A70F6E7042A04D94D4D26
:104A20002F6007F0B1F8A860FFF79AFD0422039009
:104A300003A9601C07F068F805256CE7464D062AB7
:104A400015D906222800019906F0FEFF00280ED095
:104A500006220199280007F057F806223F4928004E
:104A6000FEF7CAFB0123394A91780B439370290062
:104A70000622601C07F048F807254CE7012AA3D05E
:104A80007078FFF775FE9DE7012800D0E9E6931ED8
:104A9000334F1A2B04D87378002B09D100F014F986
:104AA000304B39001D78601C6A1E07F02DF832E784
:104AB000551E2A000199380007F026F82A49AAB2A3
:104AC0003800FEF799FB00F035F9E9E7DA281DD147
:104AD000042A00D878E7082A15D9B37972791B021D
:104AE0001343F27912041A43337A1B0613433B60D3
:104AF0003B68052231002000039307F005F80422EB
:104B0000601D03A953E7FE236370F1E7DE2800D0A0
:104B10005AE7511E012A01D10025FCE6019800F058
:104B2000CBFFF9E7A061FF1F84BD0011D461FF1F17
:104B3000FC0C000078BD0011F50C0000AC61FF1FFB
:104B40008C61FF1F5443FF1F1042FF1FD061FF1FE6
:104B5000AD42FF1FE061FF1F6509FF1FADAC000004
:104B6000D163FF1FCF63FF1FAEDE000070477047A9
:104B7000020010B5094B0A32094C92B2DA815A820E
:104B800098811882207802F03FFB0422054B012116
:104B900020781A7006F068FF10BDC046DE42FF1F85
:104BA0001A64FF1F1964FF1F013870B5042809D863
:104BB00006F042FF030928081200234B022118784F
:104BC00006F052FF70BD204B0821187806F0C4FF94
:104BD00000221E4B1A72F5E7802200241B4B1A4D4F
:104BE00052001A8108211A682878DC7206F00CFE3F
:104BF0002100287806F0E0FF012000F063FE00F0BD
:104C000075FFDFE7104B0821187806F0A5FF104864
:104C1000FFF75AF80F4B104A9B79002093800F4AF8
:104C200013808022094B5200D8721A8100F04AFE8C
:104C300000F05CFF0A4B9B78002BC3D0094A13603D
:104C400006F0DAFFBEE7C046F061FF1FC461FF1F38
:104C50001942FF1FD461FF1FE043FF1F0A42FF1FDD
:104C6000D061FF1F34F0004010B501290BD102289C
:104C700009D1054B1B78002B05D02622034B044895
:104C80005A72FFF775FF10BDF263FF1FC461FF1F6B
:104C9000C40900000300F0B50A4D8E18B14202D1DC
:104CA00052008018F0BD0C782F6824093C5D0F2756
:104CB0001C700C7801313C402F683C5D5C70023305
:104CC000ECE7C0460442FF1F0E22114B10B51A70CC
:104CD0000D23104C10492370093A043B0F486370B0
:104CE00006F012FF2D2301220D490E48E371FFF754
:104CF000D1FF01220C49FFF7CDFF01220B49FFF73D
:104D0000C9FF00220A491000FEF776FA10BDC0461E
:104D1000EE63FF1FCF63FF1F33BD0011D163FF1F81
:104D20006709FF1FD763FF1F6609FF1F6509FF1F84
:104D3000AEDE000070B5124C132220001149FEF7C0
:104D400021FB114D002817DDAB78002B14D0431C3C
:104D50002B7009236B700023001903702878290039
:104D60000130C0B206F060FF297822000139C9B2D3
:104D7000002005F0E5FD70BDFFF7A6FFEEE7C04699
:104D8000D163FF1FAEDE0000CF63FF1F10B5114BD4
:104D90001A781870002A0ED000280BD10E4B1A7802
:104DA000062A07D85423D340DB0703D50B4B1878CA
:104DB00002F02AFA10BD0028FCD0074B1B78012B0B
:104DC00002D0033B022BF5D8044B0121187806F0E2
:104DD0004BFEEFE7F263FF1F1964FF1F1A64FF1F0A
:104DE00070B54A4E4A4A4B493070022005F034FCF7
:104DF00000F0E4FEFEF704F906F086FD03224649C2
:104E00004648FFF747FF2D24030004221C70444945
:104E10000130FFF73FFF30230470424D424C437096
:104E200083702E3B062220004049EB87FEF7AAFA4A
:104E3000062813D0200006F0C7FC022809D0032161
:104E4000200006F031FD8D23E3706E3B2371193392
:104E50006371062220003549FEF7CEF9344B1B68FA
:104E6000FC335C64FFF766FF0020FFF78FFF314CD7
:104E7000314A0121314B1278207802F087F9304A0B
:104E8000304B12780021207802F080F901222E4B5D
:104E90001A702E4BDB78552B31D12D4B3B325A7289
:104EA0002C4B2D4AAB81EA812B826A8220213078FB
:104EB00006F05AFE0120404205F08EFD01204042DE
:104EC00005F02AFEFFF720F9FEF7E2FE00F0A4FC51
:104ED00001204042FEF7AAFF012006F035FCF02039
:104EE00001F010FB0121307806F0BEFD307802F0B1
:104EF000E7FA1A4806F068FEFEF7DEFD70BD642290
:104F0000174B5B7953431A000A32CBE7F061FF1F5E
:104F10006D4B0011694C00115443FF1F8C61FF1F42
:104F2000AC61FF1FDE42FF1F6509FF1FADAC000033
:104F30004464FF1F1A64FF1F3842FF1F1942FF1FFE
:104F4000EE63FF1FCF63FF1FC063FF1FD061FF1F12
:104F5000C461FF1FC4090000CE090000F261FF1FF9
:104F6000D461FF1FF8B50A0020230D001A40194232
:104F700057D0574B1B78002B50D0FFF7F1FA554B09
:104F8000554C564E99686268737A8A1ADB039A42C6
:104F900002D36160FEF790FD327A217A531EDBB2B4
:104FA000994205D1FFF768F9002000F0D9FD0FE024
:104FB0009142F9D300232372FFF788F9012000F012
:104FC000CFFD474F3800FEF77FFE390006F04CFE5C
:104FD000637A002B1FD0013BDBB26372002B1AD126
:104FE000404BDB78552B01D106F006FEE37A002B0F
:104FF0000CD000233C4A3A4FE37213883800013347
:105000001380FEF761FE390006F02EFE64237079EE
:105010005843FFF7ADFD237A013323722020684007
:10502000F8BD0BB2002B0ADA304B187806F0A4FB5F
:10503000002801D006F0F8FC80200002EFE70224EF
:10504000214206D0244B01201A72FFF79FFE200058
:10505000E5E70B071ED5FFF783FA1E4B1E491F4CD1
:1050600098684A68637A821ADB039A4202D34860DE
:10507000FEF722FDFFF72AF9FFF7FEF8012000F006
:105080006FFD00F0E3FB2368DB0701D5FEF7C6FFE9
:105090000820C4E71024214206D00D4B1B78002BBA
:1050A000D5D1FEF709FED2E70124214207D01048EE
:1050B00000F06CF806F0C8FA00F034FDC7E70424ED
:1050C000080020402142ABD0FEF7CCFEBFE7C0462F
:1050D000F263FF1FE061FF1FC461FF1FD461FF1F68
:1050E0001942FF1FD061FF1FB861FF1FF061FF1F52
:1050F000FC41FF1FF0B51B4B1B4F1B883A88040077
:105100001A4E1B4D85B09A420DD832889A420AD366
:10511000184B1A882B889A4205D1174A174B1288C8
:105120001B889A421BD0052001F042FA3B8802AA54
:1051300013803388019053802B88114D93800F4B3F
:1051400002A91B88D3800F4B2A78188802F05EFFD3
:105150000D4B08212878019A1C7006F045FD05B01A
:10516000F0BDC046BE63FF1F0E42FF1F0C42FF1F73
:105170000A42FF1FBC63FF1FBA63FF1F0842FF1FE5
:105180001A64FF1F1042FF1FB863FF1F13B50C4BBB
:105190001C78002C11D1002801D00A4B18600A4A53
:1051A0000A4B11780A4A10780A4A01920A4A009278
:1051B000002205F0BDFA200016BD1124FBE7C04611
:1051C0001964FF1FB463FF1F1864FF1F0864FF1FEB
:1051D0001A64FF1FF463FF1FF863FF1F10B5064B2F
:1051E00012201B78052B06D1044B13221988044B7F
:1051F000187801F0B9FB10BD1964FF1F1042FF1FA2
:105200001A64FF1F10B500240122114B524218707E
:10521000104B1C70104B1A8002F052F904220F4BF5
:1052200021001A700E480C3206F0FEFA10222100FE
:105230000C4806F0F9FA07220B4B1C600B4B1C7054
:105240000B4B1C700B4B1A700B4B1C7010BDC046E7
:105250001A64FF1F1964FF1F1042FF1F1864FF1F0D
:105260000864FF1FF863FF1FF463FF1FCE63FF1F77
:10527000CD63FF1F1242FF1FCC63FF1FF8B5174C11
:105280000600257806A814240078052D23D1B41F24
:10529000134FA5B21824BD421DD88D1FADB2BD421B
:1052A00019D8FA256D00AA4215D21D000D4F0A3DEE
:1052B000ADB2BD420FD80C4C26800C4C21800C495D
:1052C00000240A800B4A1380FFF714FF0A4B0421C5
:1052D000187806F041FC2000F8BDC0461964FF1F95
:1052E000790C0000750C00000E42FF1F0C42FF1FDE
:1052F0000A42FF1F0842FF1F1A64FF1FF0B50BB2DE
:105300000D0089B0002B00DB70E1A44E307806F070
:1053100033FA041E50D00378A22B00D122E1D02B07
:105320001AD0912B45D143780E2B42D19C4B8288C9
:105330009A423ED19B4A83681278052A39D10320CC
:1053400018567F2835D0984B1B68002B31D05B68EE
:10535000002B2ED098472CE08078072829D806F01B
:105360006BFB0428183F3F74A8D86378002B0CD13E
:1053700001218C4B19708D4B1A78002A5BD08C4B15
:10538000307801F003FF002855D00722854B1A70B2
:1053900051E061780029F8D1E378002B11D0854ADB
:1053A000854B1278307801F0F1FE60706378002B45
:1053B000EBD1200006F038FB80200002684009B0E5
:1053C000F0BD784B1B78022BF3D00121307806F02A
:1053D000E3F90028EAD10121307806F045FBE5E742
:1053E0006378002BD1D16F4F032807D13B78052B71
:1053F00002D101333B701EE00223FBE76F4B1A889A
:105400006F4B0293002A0BD01B78002B03D0012195
:10541000307806F0E9FB3B78062B04D1013BE9E745
:10542000029B1A70F7E7042B41D10121029B3078CF
:10543000197006F019FB5C4B1B68002BB9D01B6878
:10544000002BB6D0574A107884E76378554F002B6D
:1054500027D10622211D5B4806F056FB62895A4B74
:105460005A491A80A2895A4B1A80E3890B80052178
:10547000397058490A80584A1380228A574B1A803B
:10548000574B1B78012B09D11F2001F091F8FA220C
:10549000920042430421307806F0A6FB0022484BDC
:1054A00075E7312B00D070E70022454B1A700323BB
:1054B000A0E706220021434806F0B6F90023454A3A
:1054C00004211380444A30781380444A138006F044
:1054D00043FB0821307806F03FFBA379083B5A4292
:1054E0005341304A03331370304B1B78002B06D0E6
:1054F000334B30781A78002A06D001F085FE01225D
:10550000314B52421A8096E70121197006F0ACFA2D
:10551000F5E70821307806F01FFB6378002B00D0F8
:1055200047E72C4B2D4F0293E388029A0421138006
:10553000294B307803932389039A138063893B8036
:1055400006F02AF9002800D033E7264B1B68002B11
:1055500000D12EE7039902983A88098800881B68D1
:10556000984726E74379132B00D022E70389012BC4
:105570000AD11D4B1B78022B06D10821307806F08A
:10558000EBFAFFF72BFE14E7052001F011F80821D4
:105590000200307806F028FB0BE7C0461A64FF1FB4
:1055A000051400001964FF1FB463FF1F3842FF1F7A
:1055B0001942FF1FEE63FF1FCF63FF1FF063FF1F42
:1055C000F263FF1FC163FF1F1042FF1FC863FF1F6D
:1055D000CA63FF1FBE63FF1FBC63FF1FBA63FF1FC9
:1055E000C063FF1FB063FF1FB863FF1F8020C001AF
:1055F000014200D0E2E6CB0731D5324B1B78002BBD
:105600001DD0314E05AC3378052B1AD1023B2370E7
:105610002E4B21001B7823722D4B1B7863722D4B70
:10562000187801F057FD002809D007202A4B307068
:105630001B68002B03D01B68002B00D0984701206B
:10564000BCE60E20254B06221B7825492370254BEE
:105650001B78637002ABC01806F056FAD8E7022335
:1056600008001840194209D0174B1B78052B03D1AD
:105670001D4B188806F030F902209FE604242142D1
:1056800003D0FFF737FD200098E6082308001840F4
:10569000194200D193E6154B1C78012C03D0022C43
:1056A0000DD008208AE6124B124A134913481B8872
:1056B0001288098800880094FFF7E0FDF1E7FFF702
:1056C0008DFDEEE7F263FF1F1964FF1F1242FF1FFB
:1056D000CC63FF1F1A64FF1FB463FF1FCE63FF1F5D
:1056E0001342FF1FCD63FF1F1042FF1FB863FF1F50
:1056F0000842FF1F0A42FF1F0C42FF1F0E42FF1FFE
:1057000010B502A804880B20002C10D14968087835
:105710004978090201430C48814209D102211980CC
:105720000A4B59881170DB7800205BB2537010BDB2
:10573000074C0A20A142FAD102211980034B998813
:1057400011705B79F0E7C0466E2A0000B861FF1F58
:105750006F2A0000F7B5150008AA16884A680F4F8F
:1057600014785278120222430A24BA4214D1012238
:10577000DBB2019200962A0005F0E0FE041E0BD178
:10578000074B1B68002B07D068782A78000210436B
:1057900042425041013098472000FEBD02290000DE
:1057A0002C64FF1F30B5012503790400BFB02B42E4
:1057B00025D01449408805F02DFA28420CD0124B10
:1057C00001A95B8D00220B8002234B800F4B5B886D
:1057D0008B80608802F010FB0D49608805F01AFA92
:1057E000C0070CD50B4B01A91B8800220B8002239C
:1057F0004B80064B9B888B80608802F0FDFA3FB09F
:1058000030BDC0462464FF1F3C42FF1FB861FF1F2C
:105810001C64FF1F9642FF1F10B5074C074920006C
:1058200005F0AEF92000064905F0AAF90721054A5E
:10583000054805F067F910BDFFFF00002464FF1F55
:105840001C64FF1FA4BD00113C42FF1F10B502489D
:1058500003F054F910BDC046A5570011082110B53A
:105860000E240A4AC307DB170B405179A1430B43AF
:1058700053710223184202D051790B435371042310
:10588000184202D051790B43537110BDAD42FF1F36
:105890000A2110B50F240A4AC307DB170B40117801
:1058A000A1430B431370830703D5062311780B43E1
:1058B0001370400703D5012311780B43137010BDFB
:1058C000AD42FF1F10B5054B102419780A00A24302
:1058D000002801D022000A431A7010BDAD42FF1FFC
:1058E000662110B52024134BDA788A431979DA70CF
:1058F000A14324190C431C71542812D96020014380
:10590000197104210A43DA700222D9780A43DA7045
:105910002022D9780A43DA704022D9780A43DA7013
:1059200007E04428EDD83428EED82428F0D81428ED
:10593000F2D810BDAD42FF1FF8B50E23384C05005C
:10594000627926791A4011339E43364B6271267173
:10595000984204DD6E23E3716C3BA371F8BD324BBA
:10596000984203DA1A23E3711C33F6E700232F4928
:10597000A371E37183B259182D4889B2814224D9A9
:10598000681D0A2100B205F017FF2A4B00B29D42A4
:1059900044DC05006421280005F00EFF0A2100B256
:1059A00005F07AFE244F09B2E2797B5C1343E37180
:1059B0000A21280005F000FF0A2100B205F06CFE64
:1059C0001D4F09B27B5CA2790EE001210A4362718E
:1059D000002D1CDA5B421DB20423A371A379632D51
:1059E000D8DCFA22092DE3DC1343A3710A21280035
:1059F00005F052FE0F22114F09B27B5C1A4016438C
:105A00001F2293436279267113436371A6E7FA2339
:105A10009B009D42E2DB0123E371BBE70500FAE74F
:105A2000AD42FF1F1B4E00001DFCFFFFCB07000017
:105A3000960F00000A270000EEBD0011DEBD001128
:105A400070B51B4D04002B7900290DD08022134323
:105A50002B71632C0BDD76236A7813436B70402324
:105A6000AA781343AB7070BD7F221340F0E7230088
:105A7000093306DA58236A7813436B70AA786C23CB
:105A8000EFE70C4E002C0ADA2023644224B26B703C
:105A90000A21200005F000FE09B2735CE2E7092C40
:105AA000F6DD0A21200005F087FE00B2335CEEE748
:105AB000AD42FF1FCEBD0011F8B50A4F05003B787F
:105AC0000E00002B0CD0084C2000FEF713FC330016
:105AD0002A0020003978FEF701FD2000FEF748FC7F
:105AE000F8BDC0463964FF1FB842FF1F70B50A4EAB
:105AF0000A4D08223100280005F0A6FF002809D031
:105B0000074C31000822280005F0FEFF0921200083
:105B1000FFF7D2FF70BDC046AD42FF1F3164FF1FCB
:105B20003064FF1F102110B50C4B36201A78987185
:105B30000A401A70DA7856310A40DA706022197910
:105B400098701140223ADA71A2325A71DF3A0A4350
:105B50001A7106225A70FFF7C9FF10BDAD42FF1F30
:105B600010B5002824D0134C0A210223E05E05F072
:105B700023FE00B2FFF7E0FE0423E05E642105F09F
:105B80001BFE012100B2FFF75BFF207AFFF7A8FEA2
:105B90000320FFF763FE0020FFF77AFE064B18781C
:105BA000053843425841C0B2FFF78CFEFFF79EFF15
:105BB00010BDC046B861FF1F1964FF1F70B50025F6
:105BC0000A4C2000A571FEF795FB10233E21200012
:105BD000074AFEF783FCA84200D13E35054B200062
:105BE0001D70FEF7C5FB0123A37170BDB842FF1FF6
:105BF000BEBD00113964FF1F0200F0B501270A483D
:105C00000A4E51188B1A002B00DCF0BD08241578C1
:105C10004308684038404000805B013C58406D08B4
:105C2000002CF5D10132EDE7FFFF0000FEBD0011B1
:105C3000F0B500250F269D4200DBF0BD4C5D070945
:105C400044403440A400A05801357840F3E70000F8
:105C5000F0B589B06A460D000B000F271100103512
:105C60001C780133260024093E401670547002321D
:105C7000AB42F5D12023024AFFF7DAFF09B0F0BDAD
:105C800004BE0011F0B54E780B7889B036020C00D6
:105C9000170001901E43012A61D9954B9E4200D8FE
:105CA00077E001339E421CD1062A17D1CA788B783F
:105CB00012021A430B791B0413434A7912061A4342
:105CC0008C4B5A6100221A705A808B4A5A608B4A58
:105CD0009A608B4ADA60002009B0F0BD8822520534
:105CE000EEE7884B9E423CD182498B78002B00D056
:105CF000F6E00C2A31D10F22A3789343E278120206
:105D000013432279120413436279120613434B6042
:105D1000E279A07912020243207A00041043627AE9
:105D200012060243CA60E27AA07A1202024376485F
:105D30004A81834208D804236E49142201980B70CB
:105D400005F0E2FE1420C7E71201D21889235B0593
:105D50009A42F0D801238B70BDE7022AFAD00523BE
:105D6000EAE76A4A01239642E6D1FFF737FA052FA0
:105D70000CD9E378A2781B021343227912041A4348
:105D800063791B061343624A0393136005F034FFE3
:105D9000A1E7584D2B78002B9DD1AB78002B00D17B
:105DA000A0E02B8901339BB20093B34200D091E075
:105DB000132AD4D9CF7C8B7C3F02122120001F43B1
:105DC000FFF71AFF874200D08EE0002E3DD1E37826
:105DD000A2781B0213432279E96812041A436379FB
:105DE0001B06134303930A228B4212D1FF23A37095
:105DF000E370237163716B89002B09D1E37B227CF3
:105E00001B0212041343A27B13431B0901336B8152
:105E100000226B89002B8ED0002A67D16868370179
:105E20003818000B6B6900030390984205D968612C
:105E300005F012FDEB780133EB7068681022A11CAD
:105E4000381805F0E1FE2E8145E76F89009A7B1E28
:105E50009BB293423AD1E278A37812021A43237993
:105E600005A81B04134362796C6812061A43EB6899
:105E700000920392211D0C22049305F045FE01209F
:105E8000260004A940421036FFF7E2FE013F012F31
:105E900017D1009A0B232861824200D04CE70422DC
:105EA0001C49200005F0B0FE042203A9686805F033
:105EB000B3FEE968039AFF23914200D13CE7F73B28
:105EC0003AE73100FFF7C4FE1036DFE70923B74297
:105ED000A4D831E7009BB34200D9FCE607232BE7A7
:105EE000022329E7032327E7062325E70A2323E7DD
:105EF000FFFE0000C042FF1F00000111FFFF000075
:105F00005048593601FF0000FFFF001102FF00005A
:105F100034F00040CC42FF1F10B5034C0B000122AF
:105F2000210000F06BFA10BDD96000110B8870B52C
:105F300006000D000224162B11D92B00032209495B
:105F400000F05CFA041E0AD1074B2A881B88191C32
:105F5000934200D9111C300089B200F0EFFA200002
:105F600070BDC046056100115E64FF1F10B54A7820
:105F70000400013A0B000220012A07D80A78002AFF
:105F800004D005222000024900F038FA10BDC046B6
:105F9000336100110A7810B50B0004000220002ABA
:105FA00004D007222000024900F028FA10BDC046A4
:105FB000DF6100110A7810B50B0004000220002AEE
:105FC00004D009222000024900F018FA10BDC04692
:105FD0004562001110B5034C0B000B22210000F0AC
:105FE0000DFA10BD7562001110B5034C0B000D22A7
:105FF000210000F003FA10BDE762001110B5034C58
:106000000B000F22210000F0F9F910BD41630011CF
:106010000A7810B50B0004000220002A04D01122D7
:106020002000024900F0EAF910BDC046516300119A
:10603000002310B51322190000F0E0F910BD000094
:1060400010B5034C0B001722210000F0D7F910BD4A
:10605000A3630011002310B51922190000F0CEF936
:1060600010BD000010B5034C0B001B22210000F0F6
:10607000C5F910BDDD630011F7B584890D00060078
:106080000121002C22D000238268D3561778002BE0
:106090001EDA0C2C1AD90C3CA4B2131940880093B8
:1060A000230002F086FE431E984101307B06DB0F81
:1060B0006B703F23013C1F40A4B22870AF70AC80CE
:1060C000002C07D0B3680133AB6000210800FEBD8F
:1060D0000020EBE7AC60F8E70B7803704B88437067
:1060E0004B881B0A83700B79C3700420704704200F
:1060F000022B06D10020537811781B02009A0B4323
:10610000138070470B8803700B881B0A43700220B2
:1061100070470420009983420AD1537810781B02FB
:1061200003430B80D37890781B02034300204B80FD
:106130007047F8B50D004B7801240021461C037010
:106140002B788B4201D82000F8BD6B78B01C4F1C17
:10615000012B10D1890069184B88022233704B88BB
:10616000B9001B0A7370691805F0A6FC04360434E4
:10617000A4B2F9B2E4E7122359436B185A880431E8
:1061800032705B8810221B0A7370691805F094FC4A
:1061900012361234ECE770B5049D14001E00052B76
:1061A00001D8042070BD637812781B0213432B8042
:1061B000E378A2781B02134302226B802A71211D0F
:1061C000681D063E05F078FCB2B22A81E92AE8D8BB
:1061D0002800A11D0A3005F06FFC0020E2E7002333
:1061E00010B50A789A4201D8900010BD9A008A181A
:1061F0005488013304705488DBB2240A44709488B4
:1062000084709288120AC2700430EAE710B5110057
:10621000029C062B04D004201022142B01D010BDA8
:10622000022222714B7808781B0203432380CB782B
:1062300088781B02034363800431601D05F03CFC39
:106240000020ECE710B50C788B7804315C43E4B2A5
:1062500003702200013005F02FFC601C10BD0420EB
:10626000022B06D10020537811781B02009A0B43B1
:106270001380704710B50C000A88023105F01CFC31
:10628000208810BD70B504000D0004981100012B8A
:1062900001D8042070BD1678527812023243028071
:1062A0000200F13255701470E125002C00D10C353C
:1062B000023B9AB24280AA42EBD80231043005F088
:1062C000FBFB0020E6E70420009983420AD15378C3
:1062D00010781B0203430B80D37890781B02034392
:1062E00000204B80704710B50C000A88023105F081
:1062F000E3FB208810BD000070B501211E000420C2
:10630000049C0E400B4218D1CB40DDB28D4214D913
:106310000A49DBB2098899420FD32300EE331D707E
:106320003300580011184978165C090231430133D3
:106330002152D9B28D42F4D8002070BDD842FF1F3F
:1063400010B50C000A88023105F0B6FB208810BD9C
:1063500010B50C788B7804315C43E4B203702200F2
:10636000013005F0A9FB601C10BD10B511000298AA
:10637000032B01D8042010BD14785278043B12027C
:1063800022430280CA788C781202224342809AB259
:106390008280EB2AEED80431063005F08DFB002018
:1063A000E9E710B50C000B8803700B881B0A4370DB
:1063B0004B8883704B881B0AC3708A88043006316F
:1063C00005F07AFBA088043080B210BD0420012BB8
:1063D00003D100201378009A1370704710B50C0099
:1063E0000B8803700B881B0A43704A880230043103
:1063F00005F062FB6088023080B210BDF0B589B054
:1064000003931E4B029242000700D05A019102F002
:1064100020F81325061E2DD0029B01240370019B3A
:10642000002B04D0001903999847001984B26B46D9
:106430001B7A5BB2002B0FDA1021380002F01CFB34
:106440001925002813D130003219E1B202F066FCA0
:10645000051E0CD10C34A4B2042304AA380005A9EB
:1064600093800696948101F0AFFD051E02D03000A6
:1064700005F09AFB280009B0F0BDC0465C64FF1F20
:1064800070B505000C0000280CD00020814209D016
:1064900010222000044905F00FFB01202B78237304
:1064A0006B78637370BDC04644BE0011F0B5060042
:1064B0000D0017001C0085B002291BD000201029F8
:1064C00007D1022B07D0102B03D115E00020102C90
:1064D00008D005B0F0BD69463800FFF7D1FF2A00AB
:1064E00069460BE069463000FFF7CAFF22006946A3
:1064F000380004E0022BE9D12A003900300005F011
:106500004BFBE6E7031CF02800D9F02303200849E1
:106510009AB2013A0B80D317034006499B189B108F
:106520000B80D30F04499B185B100B807047C0464B
:10653000DC42FF1FDA42FF1FD842FF1F034B1B88BC
:106540008B4202D3024B4000C1527047DC42FF1F16
:106550005C64FF1F014B4000185A70475C64FF1FCA
:106560001722014B1A8070475C64FF1F70B505004D
:106570000E2005F009FA041E13D0D0230370002367
:106580000622837007494570033005F095FA064BE3
:106590002100DA8A62811B7E2373044B187805F090
:1065A000B3F870BD7864FF1F6864FF1F2C43FF1FA2
:1065B000262803D8024B4000C05A70470148FCE728
:1065C000DE42FF1FFFFF000070B506000C00094D02
:1065D0001C220021280005F027F9074B1E70074BED
:1065E0001C7005F019FA0123002801D000231220A5
:1065F0002B7070BD6864FF1F2C43FF1F8964FF1F51
:1066000070B505000D4C0800E260A1601022002169
:10661000656005F029F8012803D11021A06802F077
:1066200058FD10220021280005F01EF8012803D192
:106630001021606802F04DFD70BDC0466864FF1F08
:1066400070B5041E05D1002903D006220D4805F0BF
:1066500033FA0D4B1D78012D11D1002C05D10222EA
:106660001A7005F049FA280070BD00221A70074B15
:106670001B78FF2BF7D02000FFF778FFF3E700250A
:10668000F1E7C0467864FF1F6864FF1F2C43FF1FBB
:10669000030010B5002801D1002010BD00780B4A7E
:1066A000002803D15988D1821B7913761378022BE5
:1066B000F2D10023984200D103331370044B1B78AE
:1066C000FF2B01D0FFF752FF0120E6E76864FF1FB0
:1066D0002C43FF1F002911D000280CD04B79012832
:1066E00003D140225242134303E03F2213400328C8
:1066F00002D001204B7170474022F4E70800FAE70E
:1067000070B5094D0100287800280BD0074C0622EF
:10671000200005F0D1F921002878FFF7DBFF2000E9
:1067200004F0FAFF70BDC0468864FF1F6264FF1F5B
:1067300000290AD0012808D13F224B799343C02B6E
:1067400003D0403B5A425341981C704770B5174DD7
:1067500006002B78FF2B15D00A2005F015F9041E32
:1067600010D0D0230370C83B8370114B11491B78A4
:106770004670C3700622043005F09EF92100287887
:1067800004F0C2FF0C4B1B78012B0DD10B4B1B6887
:10679000002B03D09B68002B00D09847084B0421A6
:1067A0001878084A05F030F870BDC0462C43FF1F2A
:1067B0008864FF1F6264FF1F8464FF1FB064FF1FB3
:1067C000B464FF1F60EA0000014B98687047C04640
:1067D0006864FF1F014BDB68186870476864FF1F1F
:1067E000074B10B5DA68136801331360054B18784E
:1067F000FF2803D08021C90105F036F910BDC0463D
:106800006864FF1F2C43FF1FF7B50E0002F0C8F8A5
:10681000051E1CD00E4B06621F78002F00D1077892
:10682000AB791020019305F0AFF8041E0FD0D023F0
:106830000380C73B8370019BE91DC37006220430AF
:1068400005F03AF921003800E66004F05DFFF7BD7D
:106850002A43FF1F014B18787047C0468864FF1F0A
:10686000054B002805D1054B1A78054B002A00D1AD
:10687000014B18007047C0467864FF1F8864FF1FF3
:106880006264FF1F014B58687047C0466864FF1F71
:10689000024B1868431E9841C0B270478C64FF1FBA
:1068A000421E03000120152A03D9FF3B5A425341DF
:1068B000D8B27047F0B51C0000230E0085B00390DD
:1068C00002920B70029A934201D3002019E0E55C1A
:1068D0005A1CD2B2002DF8D0029851198142F4DC32
:1068E0000233DFB2A35C18000193FFF7D9FF002841
:1068F00007D0013D019A0399EBB233708A4202D16D
:10690000E01905B0F0BDDB19DBB2DBE710B50C0018
:1069100002F09EF803001220002B03D021005888BB
:1069200004F01AFF10BD000070B50E4D84006359CD
:10693000002B15D0186A002801D004F0F5FE2B5961
:10694000586A002801D004F0EFFE2B59986A0028FD
:1069500001D004F0E9FE285904F0E6FE00232B5193
:1069600070BDC0469864FF1F1C4B70B504000E003C
:10697000150099420AD11A4B1B68002B01D1122035
:1069800070BD1B68002BFAD09847F9E7154B994268
:1069900015D1134B1B68002B0AD01B68002B07D0A6
:1069A0009847002804D1104B1C70104B1D70E7E76E
:1069B00029002000FFF7AAFF0028E1D1F3E7080033
:1069C00001F0EEFF0028DAD003780320A342D7D1EC
:1069D0002900300004F0C0FED2E7C046FEFF0000F0
:1069E0009464FF1FFFFF00009164FF1F9064FF1F6E
:1069F000F7B50400808801F0D3FF0025A84203D03A
:106A00000578A08802F008F81C4E3378002B1FD0C0
:106A1000AB421DD11A4B28001978FFF777FF0028E9
:106A200018D000233370A3790820A778A688019393
:106A300004F0AAFF011E0DD0D0230370CA3B83705F
:106A4000019B477086808371280004F05DFE01E0A1
:106A5000002DE8D1A0880B4B8200D358002B01D029
:106A6000FFF762FF1721A088FFF768FDA08801F0FB
:106A700027FDA08801F0FEFDF7BDC0469164FF1F11
:106A80009064FF1F9864FF1FF0B587B01D000CAB2A
:106A90001B88070001930DAB1B88142002930EABDB
:106AA0001B88160003930FAB1B880091049310AB57
:106AB0001B88059304F068FF041E1AD0D0230370CE
:106AC000CB3B47708370C670062229000430002D2E
:106AD00011D004F0F1FF019B21006381029B00981B
:106AE000A381039BE381049B2382059BA37404F091
:106AF0000BFE07B0F0BD04F097FEECE7F7B500938E
:106B000008AB1B8807000C200D001600019304F051
:106B10003BFF041E13D0280001F042FF00280FD0D5
:106B20000078D0232370C93BA370009B21002381F0
:106B3000019B6770A580E680638104F0E5FDF7BDE9
:106B4000014B1878EDE7C0462C43FF1F13B5040036
:106B500064890389C2888188C0780094FFF7CEFFDA
:106B600013BD000010B5044C2068002803D004F0C9
:106B7000DBFD0023236010BD9C64FF1FA122F0B544
:106B8000818892004A43384B384F1B6804009B1899
:106B90009D2292009B18827989B01A603B68002B75
:106BA0005FD01D78324B1B68002B04D05B68002B34
:106BB00001D000209847260008363100E079FFF721
:106BC000B7FD237DE0710200E0780493638A290019
:106BD0000393238A0293E3890193A38800933300EC
:106BE000FFF752FFE378002B0BD1E289A379A1884C
:106BF00002920196E27928000092012201F0DAFE69
:106C0000E0703B68002B20D0FFF7ACFF194D2878CF
:106C100000281AD0184B1978FFF778FE002814D0F6
:106C20002B78E67808200793A78804F0ADFE011EB4
:106C300009D0D0230370CA3B467083708780867169
:106C4000079804F061FD00232B701721A088FFF73F
:106C500075FCA08801F034FCA08801F00BFD09B0A0
:106C6000F0BD064B9DE7C0463409FF1F9C64FF1F23
:106C7000B064FF1F9164FF1F9064FF1F2C43FF1F30
:106C8000F8B5070008000E0001F08AFE041E18D0B7
:106C90002620FFF78DFC051E00D12578062004F084
:106CA00073FE041E0DD00021062204F0BDFDD0238A
:106CB0002370C23B21006770A370A680E8B204F085
:106CC00023FDF8BDF0B585B001930AAB1B78070032
:106CD00002930BAB1B7808000D000092039301F0A8
:106CE0005FFE061E22D0102004F04EFE041E1DD0B2
:106CF0001022002104F098FD2620FFF759FC0028FF
:106D000000D13078D0232370C13BA370009B2100B9
:106D10002372019B67706372029BA580A372039B21
:106D2000C0B2E3720C9BE36004F0EEFC05B0F0BD72
:106D3000F7B50D00019001F033FE071E20D00E20A4
:106D400004F022FE041E1BD02620FFF731FC061E95
:106D500000D13E78D0232380C53B0622A370F91DC5
:106D6000E01C04F0A9FE019B2A0063810123DD40A1
:106D70001A401D40210022736573F0B204F0C4FC78
:106D8000F7BD0000F0B585B0029010000D001700AF
:106D90000A9E039301F004FE041E31D0029B002BD7
:106DA0002ED1039B02795B0724D5122313430422BF
:106DB000002E08D10B99002905D10C99002902D188
:106DC0000D9900291AD01A430D9B2271002B00D077
:106DD000C9E0002E00D1CFE0002D00D0CCE0606AE9
:106DE000002801D004F0A0FC1C21300004F00CFEAF
:106DF000606205E002239A430E33D7E79343237181
:106E0000654BBA00D458002C00D1AAE0002E10D057
:106E1000236A002B03D11C2004F0AEFD20625E4BE0
:106E2000BA00D358186A002803D01C22310004F09D
:106E300043FE0C9B002B12D0574CBB001D596B6AB4
:106E4000002B03D1162004F097FD6862BB00E358C5
:106E5000586A002803D016220C9904F02DFE0D9BD1
:106E6000002B11D04C4DBC006659B36A002B03D1E6
:106E7000142004F081FDB0622B59986A002803D0D9
:106E800014220D9904F018FE380001F089FD051E4A
:106E900067D0414BBA00D358002B62D01A6A342015
:106EA000002A00D11C389A6A002A01D0143080B21E
:106EB0000B9A002A01D01C3080B25B6A002B01D0F3
:106EC000163080B204F060FD041E4AD01822002162
:106ED00004F0AAFC2620FFF76BFB0190002801D1EB
:106EE0002B780193D0232370029B200063700A2328
:106EF000294EA370039BBD00A371AB59A780196AEB
:106F00001830002905D01C22A06004F0D5FD200017
:106F100034307359996A002907D0030014221433BE
:106F2000E060029304F0C8FD02980B9B002B08D090
:106F300003001C221C330B992061029304F0BCFD5A
:106F400002987359596A002903D01622606104F02F
:106F5000B3FD6B462100187904F0D6FB3800FFF72B
:106F6000E3FC05B0F0BD10220D9B0D991B69A01824
:106F7000236204F0A1FD2CE70B9B002B00D13FE71F
:106F8000012D00D03CE7606A002801D004F0CCFB62
:106F90001C210B982AE7C0469864FF1F10B5044CCB
:106FA0002068002803D004F0BFFB0023236010BD3D
:106FB0008C64FF1F0B4B07B51A68002A01D1002013
:106FC0000EBD6946531C012012780731FFF772FC91
:106FD0000028F4D002780123100018401A42EED0A5
:106FE000EEE7C046A864FF1FF0B51F4F01203B68C5
:106FF00087B0002B25D09B78059300F0B3FB0028C9
:1070000021D00A20FFF7D4FA04000B20FFF7D0FAB2
:10701000164B05001E78731E9E413B68F6B2191D83
:10702000D878FFF757FB3B682900DA7A04330392DC
:107030009A7901930292009033002000059A04F09F
:107040002BFD07B0F0BDFFF7B5FF002805D00620E7
:10705000FFF7AEFA04000720D8E70820FFF7A8FAE8
:1070600004000920D2E7C0468C64FF1F8864FF1F1C
:1070700070B50A4E040033780D00FF2B0DD00420AC
:1070800004F082FC011E08D0D0230370CE3B457073
:107090008370C470307804F037FB70BD3C43FF1F31
:1070A00070B5040006200D0004F06EFC011E0AD02D
:1070B000D0230370CD3B8370054B44701B688580E3
:1070C000187804F021FB002C01D0FFF767FF70BD9A
:1070D0008C64FF1FF8B5264F06003B680D00112495
:1070E000002B05D10522234B1B78134202D1122419
:1070F0002000F8BD204A10241268002AF8D0127827
:10710000002AF5D0DB0719D52B789A1E012A1AD848
:107110000C2004F031FC132438600028E8D0002350
:107120000A22437029000670023004F0C5FCFFF704
:107130005BFF041E0AD0FFF731FFD9E700F012FB16
:107140000028E1D1E4E7002BE2D0D0E70B4B1B781D
:10715000032BCDD11D20FFF72BFA094B18800028F7
:10716000C6D0084B04211878074A04F04DFBBFE74E
:107170008C64FF1F8964FF1FA864FF1F8864FF1FC2
:107180008664FF1FB464FF1F60EA0000F7B5019337
:10719000194B14001A78052306000F0012201A421A
:1071A00021D0012920D1154B1D68002D1BD00220B4
:1071B0001F2C18D8002C02D0019B002B13D0104B91
:1071C0001F221E706E1C0021300004F02DFB01995F
:1071D0002200300004F070FC310020002C70002FE1
:1071E00006D004F061FCFEBD064B12201D68DCE7F2
:1071F00004F01AFDF7E7C0468964FF1FA864FF1F6B
:107200003C43FF1FA464FF1FF8B50F4E12243368E0
:10721000002B17D01B780F3C834213D100250B4F56
:107220000221387804F098FC094B042138781D803D
:1072300004F092FC074B28001D8033685C7004F05A
:1072400053FA04002000F8BD8C64FF1FB464FF1FD4
:10725000A064FF1F8664FF1F70B5012823D11B4C5B
:107260002388002B03D01A4A1578002D07D0194B1C
:107270001B68002B02D01878FFF7C6FF70BD3B2BB0
:1072800002D93C3B2380F9E7134E0221307804F009
:1072900063FCFA222388920002215A43307804F0DA
:1072A000A3FC2580EAE70B4B1B68002BE6D00B4BB9
:1072B0001B785B07E2D5084B0221187804F04CFCE0
:1072C0000022024B1A80FFF769FED7E7A064FF1F78
:1072D0008464FF1F8C64FF1FB464FF1F8964FF1F59
:1072E000F8B51E4D2868002803D004F01DFA0023CD
:1072F0002B601B4E3068002803D004F015FA0023E1
:107300003360184F05243B7818002040234221D0D9
:10731000154800F02BFA3B78234213D0202004F0CC
:107320002BFB2860002813D02022002104F07CFAD7
:10733000202004F021FB041E306005D02022002113
:1073400004F072FA002004E0286804F0EDF92C60E3
:107350001320F8BD00F00AFAF4E7C046A864FF1F46
:10736000A464FF1F8964FF1F3043FF1F10B50A4C40
:1073700023681A1E0ED0002808D10130587004F07E
:10738000B3F9002805D02368002B02D00021FFF7B5
:1073900087FE0122100010BD8C64FF1FF7B5274E39
:1073A000050033680191181E21D05C78244F012C10
:1073B00030D1FFF7FFFD002825D02000FFF7F8F8B7
:1073C0000400412814D91F4B022118781E4A04F0EA
:1073D0001BFA1E4B3C3C1C80022233685A703B78DF
:1073E000002B14D128000199FFF75AFE0120FEBDA1
:1073F000FA2292004243002AEED0124B0221187862
:1074000004F0F2FBE8E7FFF7D3F80200F3E700230C
:107410003B70EBE73B78002BE8D1032004F0B4FA93
:10742000011E08D0D0230370CC3B457083703368B5
:10743000187804F069F9FFF7B1FDD7E78C64FF1FF6
:107440008464FF1FB464FF1F60EA0000A064FF1F94
:1074500010B51749838802008B4220D011D81549F6
:107460008B4217D0144900205B1899B2012907D824
:10747000926811785A425341D8B2FFF7F9FD0120C2
:1074800010BD0E4A00209B1807229BB29A42404131
:10749000C0B2F5E783681878FFF768FFF0E7836804
:1074A00099785A78090218781143FFF777FFE7E7D0
:1074B0000A20000006200000F8DFFFFFAFDFFFFF1B
:1074C000014B18707047C0463D43FF1F10B5064C76
:1074D000207001F041FA207804F07EF9052120782F
:1074E00000F062FD10BDC046B464FF1F0BB273B55F
:1074F0000D00002B00DBC4E0884B187804F03CF949
:10750000041E0ED00378912B0FD0A22B00D1A1E046
:10751000834B1878FF2852D0210004F0F5F800289A
:107520004DD180200002684076BD43780F2B76D085
:1075300013D8052B70D00E2BEAD18088794B984256
:107540002BD8794B98421BD8784B9842E0D1A3684E
:107550001878591CFFF774F838E03E2BD8D183789F
:10756000032B74D06CD8012B6ED0022BD0D1704B72
:107570001B68002B23D05B68002B20D098471EE0AF
:107580006C4BC0180C28C3D804F04EF81DC2C215AD
:107590000BC20B0B0B3223C23C00674BC0180728F1
:1075A000B6D8664B1B68002B09D01B68002B06D091
:1075B000200098470AE0A3681878FFF7C7F8200072
:1075C00004F032FAADE7A068FFF762F800289FD018
:1075D000F5E7A3681B78002BF1D0554B1B68002BF7
:1075E000EDD01B68002BEAD0210055489847EDE705
:1075F0004F4B1B68002BE2D01B68002BDFD0210013
:107600005048F3E7504B1B68002BD8D05B68002B29
:10761000D5D021004348E9E7FFF7EAF9CFE78088B2
:107620004A4B984203D04A4B984200D070E7464BF1
:107630001B68002BC3D05B68002BC0D02100D5E7AE
:10764000153B012BBBD963E7FFF798FAB7E7FFF7C4
:107650007DFAB4E73F4B1B78042B07D100236A4621
:1076600013800179408800F0C5FCA8E7364B1B6801
:10767000002BA4D05B68002BA1D0010036489847AE
:107680009DE7012421420AD0294B1B68002B04D01E
:107690005B68002B01D000209847012043E78B074F
:1076A0000AD5264B1B68002B04D05B68002B01D049
:1076B00020009847022036E70421280008400D42A8
:1076C00000D131E7254E3388002B21D0013B9BB2FE
:1076D0003380002B1AD1FFF7DBF800280AD0204BAB
:1076E0001C70164B1B68002B04D05B68002B01D06C
:1076F00020009847FFF7C6F8694601F001FD68468B
:10770000FEF7FEFF1D20FEF753FF308004200AE73E
:10771000024B187804F020FAF8E7C046B464FF1F63
:107720003D43FF1F0E200000012000000910000053
:10773000AC64FF1FFEDFFFFFAFDFFFFFB064FF1F82
:107740000C2000000B2000009464FF1F0D2000009F
:10775000132000008964FF1FFFFF00008664FF1FE5
:107760008464FF1F10B501F09BF910BD014B186038
:107770007047C046B064FF1F0B880020162B01D84D
:1077800017230420014A13807047C0465E64FF1F20
:1077900000207047074A03001188814207D0918872
:1077A0000020994202D1013080001018704700205B
:1077B000FAE7C046BC64FF1FF0B58F7806000D00E5
:1077C000C5B01E2F15D1FFF7E5FF051E03D100241C
:1077D000200045B0F0BD00223B003100C07800928F
:1077E00000F0B2FB0400A81C00F0D2FBFF23EB70FA
:1077F000EEE7264B062403931B78FF2BE8D0182FC7
:10780000E6D87B08224A013BDB0002929A58944654
:10781000002ADDD0029AD3185B68002BD8D00878F4
:10782000002802D14B78012B02D10624122FCFD190
:1078300007AFAB88697800976446AA68A047041E22
:10784000C6D1AB78029A5B08013BDB00D318390044
:1078500030005B689847041E0BD1AB78042BB6D080
:10786000039A310010782200009700F06DFB0400AD
:10787000AEE76A78002AABD1AA7805A93B880871DF
:1078800030000A704B80FEF747FBA0E74043FF1F24
:1078900054BE00111D4B37B5050098420BD000298E
:1078A0000AD1FFF777FF002805D11948FFF772FFCB
:1078B000002800D0058037BD01291AD1FFF76AFFE3
:1078C000041EF8D001235B420380A378FF2BF2D083
:1078D000FE2B07D00023E0781422009329001E33EA
:1078E00000F032FBA01C00F053FB01235B426380DD
:1078F000E1E70229DFD1013901F0BEF80028DAD131
:107900002800FFF747FF041EDFD1D4E7FEFF000089
:10791000FFFF0000022210B5074B52421A800748B1
:1079200001325A809A80DA8000F07EFA044801F031
:1079300025F8002010BDC046BC64FF1FB9770011B8
:10794000957800110388F7B50400002B02D10225B9
:107950002800FEBD42680221137825485268FEF7D0
:10796000A5FD00282ED0234F01253A88002AEFD00C
:10797000802321885B0201259B1A9942E8DC0C20B8
:1079800003F0FAFF061E31D03B8822889C46002374
:107990001800019561469DB2491989B2AA421BD8C7
:1079A000002801D062443A8000233000082208C039
:1079B000210004F081F8104A1368002B13D1002530
:1079C0001660C5E76268022113780C485268FEF71A
:1079D0006DFD0028C7D1BAE760681D0140194181DB
:1079E00001330198D6E71A001B68E6E71325AFE7D5
:1079F000C2BE00113E43FF1FB864FF1FC0BE00118E
:107A0000014B18707047C0464043FF1F14230A0003
:107A100010B51A40194204D00122102101F048F893
:107A200010BD4B06F9D4012088434000F8E710B59B
:107A300014008B0604D50122102101F039F810BD85
:107A400008230A001A40194202D14BB2002B0FDA68
:107A5000102101F02DF8002808D02300F2331B7804
:107A6000002BECD0F1342378012BE8D10020E6E79D
:107A700003208907FAD4E2E7F0B51F00184B85B060
:107A80001C68019002910392002C27D1200005B0C0
:107A9000F0BDA5683301ED186B89019A934211D3AB
:107AA000029A93420ED8002F04D10A9B002B10D1CA
:107AB0002C00EBE73B002978039A6868FEF7F6FC98
:107AC0000028F2D10136B6B2A388B342E1D82468C7
:107AD000DAE7A3680A9A5B891380E9E70026F3E7EF
:107AE000B864FF1F37B50C000A884988012391420A
:107AF00017D3002A15D0651D23792A0002210A48D0
:107B0000FEF7D4FC102300280BD02379618820884D
:107B100000242A000094FFF7AFFF0A23A04200D000
:107B2000230018003EBDC046C2BE001113B50A00B6
:107B300008884988012388420BD8002809D00024EE
:107B4000137905320094FFF797FF0A23A04200D073
:107B50002300180016BD13B50A00088849880123C0
:107B600088420BD8002809D00024137905320094EC
:107B7000FFF782FF0A23A04200D02300180016BDA1
:107B8000F0B58BB003904A8808880E00012382422A
:107B900055D3002853D00023012704AC23700022C2
:107BA000718813000092FFF767FF051E3ED0207812
:107BB000002835D12B78022B18D167706A89830091
:107BC0000130E31880005A8069680222201803F00F
:107BD00073FF23780133DBB22370042B19D93B00E8
:107BE0006889013080B2002BD9D01FE00223637076
:107BF000122358436A89231804305A806968102276
:107C0000201803F059FF23780133DBB22370002BD7
:107C1000E5D10C4A6B899B185A425341DBB2DFE72E
:107C20006378012BE4D12B78022BC7D022780A236A
:107C3000002A04D021000398FEF798F900231800C9
:107C40000BB0F0BD0100FFFF0F4BF0B5040018684A
:107C5000002816D083685D89A54207D88288AE18AF
:107C6000B44203DA12019A18934201D10068EFE797
:107C70001E005F891036A74204D1002900D00D8074
:107C80001800F0BD3300EFE7B864FF1F70B50500C2
:107C90000C0008880021FFF7D7FF03000120002B0C
:107CA00004D022002800197AFFF7C1FE70BDF7B595
:107CB0000C00002501902300EE331B78AB4201D865
:107CC00000200AE06B00E65A00213000E718FFF7B9
:107CD000BBFF002802D126800130FEBD017A019849
:107CE000FFF794FE002802D03B882380F5E701359A
:107CF000EDB2E0E710B5040008880021FFF7A4FF0B
:107D000003000120002B03D02000197AFFF77EFE2C
:107D100010BD0000054B1B68002B01D1180004E0CA
:107D20009A6852898242F6D198887047B864FF1FDA
:107D3000F0B50E27002687B0039302ABFF183E80F4
:107D400005001F4B40891400984207D02B78013062
:107D500000976A6880B2FFF78FFE060002212B7839
:107D600018486A68FEF7A2FB00280FD06C89200033
:107D7000FFF7D0FF002802D0013C0419A4B2039BF6
:107D8000002B00D01C80300007B0F0BD02212B7802
:107D90000D486A68FEF78AFB0028E7D102212B789C
:107DA0000A486A68FEF782FB002807D0002EDED062
:107DB0003B88A342DBD17489013CDFE76C89DEE7B5
:107DC000FFFF0000C2BE0011C0BE0011BEBE001108
:107DD00010B50C00FFF7DEFC03000220002B0AD0D8
:107DE000002C00D023609B781720FE2B03D0013895
:107DF000FF2B00D1002010BD73B50D0001A90400B8
:107E00001600FFF7E5FF172805D0002E04D1290042
:107E10002000FEF727F976BD01221021200000F096
:107E200047FE0028F3D0F6E7014B18607047C046C4
:107E3000C864FF1F37B56B469D1D01000400022278
:107E4000280003F061FE2B88B02B0ED12379122B72
:107E500009D12300FA331B78012B06D10121608858
:107E600000F0E0F801E01B2BF8D037BD10B5054B52
:107E70000421187000F098F8FFF74CFDFEF770FB36
:107E800010BDC046CC64FF1F0020F0B50BB20F0040
:107E900087B0834234DA274B187803F06DFC051E57
:107EA0002BD00378A02B25D103AE3100FEF7E4F8E8
:107EB000041E0BD1B378DB0724D51F4B06341B6897
:107EC000002B03D03100688898470400A868002878
:107ED00001D003F069FE002C08D1184A039B13401F
:107EE000174A934206D0B3781B2B03D00121688830
:107EF00000F098F8280003F097FD802000027840F9
:107F000007B0F0BD0F4B1B68002B10D03100688804
:107F10009847041EDAD07378002BD7D1B27801A924
:107F20000A704B800C716888FDF7F6FFCEE70624D7
:107F3000F1E7C046CC64FF1FC464FF1F00FFFF00D1
:107F400000011200C864FF1FF7B50190FC200D006E
:107F500017001E0003F018FD04001320002C12D09F
:107F6000B02320002370089BF4226770658026717F
:107F70000830002B08D0190003F09EFD2100019865
:107F800003F0C2FB0020FEBD089903F04DFCF5E7AD
:107F900010B5041E06D00078FD2803D803F02CFC91
:107FA000FF23237010BD00000A1F93B210B5040018
:107FB0000220032B05D882400020024BD1529B188F
:107FC0009C7010BDEC64FF1F0B8870B5043B04006F
:107FD0000D000220032B0BD80121200000F04CFDE6
:107FE00003001420002B03D02900200000F0DEFB4A
:107FF00070BD000007B51300034A00920A0001217A
:1080000000F02CFC0EBDC0463182001107B5019274
:1080100003220092024B0A00122100F049FC0EBD1F
:10802000AF82001107B56B4601AA11800449D880C0
:1080300008780633012802D1190003F095FC07BD2A
:10804000CD64FF1F0C4B10B518700023FF210B4AA5
:108050001380138193819380094A53801370517266
:1080600093819372D174D3821375517703F02CFBF3
:1080700000F0FCF910BDC046FC64FF1FEC64FF1F5C
:10808000CE64FF1FF0B58DB06B46002003910C222B
:108090009B5E834200DBB0E05D4B187803F06CFB25
:1080A000051E00D1A4E00378902B00D09DE006AF20
:1080B00001004688380000F013FA796804000029AE
:1080C00000D19CE03B88052B6ED13B89032B1CD94A
:1080D00005AC200000F0A2F86288172A61D839891F
:1080E000131D994231D17968237804310291D9075F
:1080F00038D5607800F08EF9071E06D00023037192
:108100002378012B08D0132B23D0A868002800D196
:1081100078E003F049FD75E06288029909A800F053
:10812000A6F80290380000F08BF909AA2378387A73
:108130000192002231000092029A00F012F93800F8
:1081400000F064F9029B002BDFD0300000F080F9D2
:10815000DBE70378032BD8D16288029909A800F0E5
:10816000D6F8DEE7122B13D1029909A800F0B5F872
:10817000021EEAD127498B88002BC6D0887909A92D
:108180002378019161780091310000F0EAF8BCE7B2
:10819000002302AA93833000617809AAFFF72AFF1F
:1081A000B3E71D4B0993F6E7042B02D09A1F012A6F
:1081B000ABD8184A043B9B00995A0029A5D0D21885
:1081C000907831003A0000F0AEF800289DD13B884D
:1081D000042B03D001213000FFF724FF012C04D130
:1081E000A868002801D003F0DFFC280003F01CFC85
:1081F0008020039B0002434018000DB0F0BD012811
:1082000000D182E701213000FFF70CFFEDE7C04607
:10821000FC64FF1FEC64FF1F010017000B78037064
:108220004B784370CB788A781B02134343807047A6
:108230000A88030002700A88120A42700A88012A1A
:1082400006D14A8882704A88120AC2700420704798
:1082500002208242FBD14A8804309A704A88120A6E
:10826000DA708A881A718A88120A5A71EFE710B593
:108270000400012082420CD94B780A781B02134378
:108280002380834206D1CB788A781B021343638014
:10829000002010BD022BFBD1CB788A781B02134340
:1082A00063804B790A791B021343A380F0E70B88A4
:1082B00003700B881B0A43704B8883704B881B0A22
:1082C000C3708B8803718B881B0A4371CB888371C1
:1082D000CB881B0AC3710820704703000120082ABD
:1082E00014D14A780878120202431A80CA78887832
:1082F000120202435A804A790879120202439A8094
:10830000CA798879120202430020DA80704710B5DA
:1083100004000120022A05D100204B780A781B02B4
:108320001343238010BDF8B5060010200F00150080
:1083300003F02AFB04000120002C0ED0A0230C2205
:10834000290023806780201D002D07D003F0B4FB97
:108350002100300003F0D8F90020F8BD03F064FAE2
:10836000F6E7F7B51E00009008AB142017001D7843
:10837000019103F009FB041E12D0A2230370019B9C
:1083800047704380099B057146710C220830002B11
:1083900007D0190003F090FB2100009803F0B4F916
:1083A000F7BD099903F040FAF6E737B5041E0FD080
:1083B0004388002B0CD00025C1881323007A172294
:1083C00001950095FFF7CDFFFF236580637225704F
:1083D00037BD000010B50C4904004A88002A09D0B6
:1083E0008B89002B05D00020CB8A0222834201D04A
:1083F00010BD012213000A20434300204032C8541C
:10840000C81842800472F3E7CE64FF1F0023438044
:1084100003707047094B00211A0010B55C88002CCE
:1084200006D01C79844203D10A234B43D01810BDD7
:1084300001310A330329F1D10020F8E7CE64FF1F90
:1084400010B50400407A03F0D7F9FF23637210BD22
:108450007047043010B580B203F0C6FA002803D08C
:108460000421494203F048F910BD000070B5002511
:10847000104CA0682580A581A580A84202D003F0F9
:1084800093FBA56000250C4C0C4B606D1D802300F8
:1084900058331D70A84202D003F086FB65650025A5
:1084A0006068002801D003F07FFB013508340A2DF5
:1084B000F6D170BD9465FF1F3865FF1F8865FF1FEB
:1084C00070B5041E09D1054D2880A881A880A86830
:1084D000002802D003F068FBAC6070BD9465FF1FFC
:1084E000F0B54B8885B00193002343600A790500FD
:1084F0000F00022A00D07BE0CA88032A17D98B68B4
:108500005E7819783602DC78D8790E4399781B7A30
:1085100024021B020C43034353495BBA0B80331DF7
:1085200093421ED1042C04D0631F022B0ED90120CC
:1085300015E0019A4D4B1201D35A002B06D0019839
:10854000FFF7BEFF4A4A1369013313610421B8687B
:108550002E812C80494203F0CFF86860002005B0DE
:10856000F0BD434D042C06D0631F022B0FD9EB68DE
:108570000133EB60DBE7019A3C4B1201D35A002B2D
:1085800005D00198FFF79CFF2B6901332B61374B16
:1085900030000293019B029A1B0101930023019971
:1085A0008C468B52130063449C8003939E81FFF79B
:1085B00050FF039B041E986016D00421B8684942FE
:1085C00003F09AF8FA880100043A200003F074FAE4
:1085D0000199029AFB888A5A043B9B18029A8B5293
:1085E0002B6801332B60A2E7AB690133AB619EE7D7
:1085F0001E4B0293019B1E01029BF35A002B2DD0B0
:1086000002998C19A068002828D0012A26D1FA885E
:108610009B189BB27352A189994217D39B1AC01819
:10862000B96803F049FA029BA289F35A934200D039
:108630007DE700222B81A3882B80A3686B60029BBF
:10864000F2520B4A53680133536070E7084A93684B
:10865000013393600198FFF733FF68E7044A5369D9
:1086600001335361F6E7C046FE64FF1F9465FF1FA8
:108670000465FF1F70B5051E15D10B4C0B4B188000
:10868000230058331870606D002802D003F08CFA74
:108690006565250050356068002801D003F084FA34
:1086A0000834AC42F7D170BD3865FF1F8865FF1FE5
:1086B000F0B51700A12285B0920001934243394BD7
:1086C00006001B680C009B18D933FF331D78FDF79B
:1086D00041FF0430854204DD3000FDF73BFF0430EC
:1086E000C5B2BD4207D33A0000213000019B03F020
:1086F000CBF905B0F0BD2900380003F00DFA2300D6
:10870000C6B250331E700393019B29006365380085
:1087100002F0D2FFCBB20293002B02D0039B0136B2
:108720001E7000262300503303931B78B34204D8F5
:10873000606D002831D10020DBE7029A2800002A72
:1087400004D0013B1000B34200D02800F700E71925
:10875000387003F081FA786000280ED03A780199D9
:1087600003F0AAF9019A3B780136D3180E4A019317
:10877000D369F6B20133D361D4E7039B1870606507
:10878000A74205D1084A1320D36A0133D362B0E768
:10879000606803F009FA0834F2E703F005FA0023F1
:1087A0006365C8E73409FF1F0465FF1FF7B50D00B7
:1087B00007000421686802F09FFF2B890400037002
:1087C0002B891B0A43702B8883702B881B0AC3706C
:1087D0002E8902250436F6B2F42E15D81B4B9F4283
:1087E00014D10C2003F0D0F81135011E0CD09023C9
:1087F00003708E3B0371043B4380154B8460C6803D
:10880000187802F081FF00252800FEBD5C237B4321
:10881000104AD3180093583301931B78002B0FD1C3
:108820000300320038000099FFF742FF019B05006A
:108830001B78002BE8D13800009903F055F9E3E7E5
:10884000054A0725536A01335362DDE7FEFF000046
:10885000FC64FF1F3865FF1F0465FF1FF0B587B07C
:10886000009017200F0016000193FFF7F2FD13256B
:10887000041E19D00C98031E02D00199201D9847A0
:10888000030AE370052302AAA070043090812770C8
:108890000098667003A993800494FFF787FF051E74
:1088A00002D0200003F080F9280007B0F0BD0000DE
:1088B000F0B587B01F000CAB1B7803910593012125
:1088C0000DAB06001C78049200F0D6F814250028A1
:1088D00021D02000FFF77EFD0135041E1BD0114979
:1088E000059B0A7803700132D2B2131EC68001D1F3
:1088F00001231A000B7022713000049B039900972A
:10890000FFF7ACFF051E09D1230021000648074AE6
:10891000093302F0D1FF280007B0F0BD00236380C7
:108920002370F8E70065FF1FAB830011307500006E
:10893000F8B505000E00064C064F2368002B02D048
:108940003100280098470434BC42F6D1F8BDC04637
:10895000A465FF1FB865FF1F0123064A5B425380D1
:10896000002313715362044A136053609360D36011
:1089700013617047B865FF1FA465FF1F0200002345
:1089800010B506499C000859002801D1625010BD5D
:108990000133052BF6D11320F9E7C046A465FF1F6C
:1089A000034A5388181A43425841404210407047C6
:1089B000B865FF1FF0B585B002930AAB1F780CAB0A
:1089C0001B88009008000E0001920393FFF7E8FF58
:1089D00005001120002D1BD10E48FFF7E1FF040018
:1089E0001520002C14D006220B99A771E01D03F06E
:1089F00063F8019B30002371029B29006371009B87
:108A000066802370039B6562E381FFF791FF280076
:108A100005B0F0BDFFFF000010B5FFF7C1FF040077
:108A20000220002C12D060880121FFF781FF606ACC
:108A3000002801D002F078FE28220021200002F058
:108A4000F3FE012300205B426380207110BD000013
:108A500030B5074A074C5588010013780020A5421D
:108A600004D05B1A59424B415842104030BDC046B9
:108A7000B865FF1FFFFF0000084A10B501230C0076
:108A8000904208D0FFF78CFF031E04D003792340E7
:108A90005A1E9341DBB2180010BDC046FEFF000015
:108AA000024B1879431E9841C0B27047B865FF1F4A
:108AB00070B504000D001600FFF772FF002804D106
:108AC0000D4B9C4200D0143070BD416A03790520E3
:108AD000002907D012221A40102A02D10520002EA8
:108AE000F2D10F20DB06EFD5897E0C20A942894107
:108AF000494249420840E7E7FEFF0000030010B585
:108B0000002800D110BD0348034A41889142F9D0A2
:108B10009847F7E7B865FF1FFFFF0000002330B557
:108B2000C45CCD5C6C40D4540133102BF8D130BD03
:108B30000F23002210B5C45C64002243CA54C25CF7
:108B4000D209013BF7D210BD0200010010B520325E
:108B5000103102F031FF10BDF0B58BB00390102042
:108B600005931700049102F007FF0090102002F017
:108B700003FF009B13240190002B05D000280CD18B
:108B80001324009802F0D0FD019B002B02D01800A6
:108B900002F0CAFD20000BB0F0BD102002F0ECFE88
:108BA0000600102002F0E8FE13240500002E00D17C
:108BB000AEE0002819D01022002102F035FE32006C
:108BC0002900039802F0F8FE041E0ED133787F2BA3
:108BD00051D830000099FFF7ABFF009B1B787F2B2B
:108BE00053D801990098FFF7A3FF300002F09CFDD5
:108BF000002D02D0280002F097FD002CC1D11020DA
:108C000002F0BAFE0600102002F0B6FE0290002E1E
:108C10007CD0002878D03A000F32230001251211B1
:108C200005D00F333B4015B25A4253411BB26A1E66
:108C30001201002B33D0049BD2B298180099029AEB
:108C4000FFF76CFF013D10220021300002F0ECFD27
:108C5000ADB2049F2D017D19AF4242D0002C33D01C
:108C6000300002F061FD029B002B00D189E7180063
:108C700002F05AFD85E729003000FFF759FF280070
:108C80002549009AFFF74AFFA7E729000098FFF758
:108C90004FFF28002049019AFFF740FFA5E70F2169
:108CA0000F4004998A18D9B28F4208D9D15C06A81E
:108CB00019540133102BF6D1029A0199C0E7791AA1
:108CC00048424141C901F2E73900300006AAFFF7E6
:108CD00025FF3200039806A902F06EFE103704004B
:108CE000BAE7002CBCD13000029906AAFFF716FFA4
:108CF000320006A9039802F05FFE0822040031004A
:108D0000059802F0D9FEABE71324A9E71324AAE7DC
:108D1000002800D06EE733E7C8BE0011F0B58BB075
:108D20000F0016000225009000283FD0002A3DD0F9
:108D30000B1DDBB21800029302F01EFE1135041E5B
:108D400034D0FDF747FD05003A000099201D02F0E0
:108D500083FCEBB20393E3702B0CDBB22F0A00937E
:108D60006370FFB22B0E2370A7700193FDF72CFDEB
:108D70001022010006A802F06FFC2100029A04AB49
:108D800006A8FFF7E9FE051E0DD1039B08223370EC
:108D9000009B04A9B370019B7770F370301D02F043
:108DA0005BFCFDF71DFD200002F0BEFC28000BB0AF
:108DB000F0BDF0B58FB00D00149E039004920593A2
:108DC000002A03D1022420000FB0F0BD002EF9D0FC
:108DD0000398FFF7E5FD1424071EF4D0727833786A
:108DE00012021A43B3781B041343F27812061A4393
:108DF000036A0192934201D30133E3D1002D03D0E2
:108E00003B7901249B07DED50822002106A802F049
:108E10000BFD059B13240433DBB21800029302F010
:108E2000ABFD051ECFD0059A0499043002F014FC66
:108E300004223100280002F00FFC3900102210310A
:108E40000AA802F009FC2900029A06AB0AA8FFF75B
:108E500083FE041E0FD1082206A908A802F0FCFB1D
:108E60000822311D08A802F097FE012807D10199B8
:108E70000398FDF7C9FC280002F056FCA3E7012483
:108E8000F9E7000070B51C4C05002368181E10D0CF
:108E9000002D14D11A78002A0CD1981C083202F047
:108EA0000BFE02F021FD0135002808D123681D705A
:108EB000012070BD0A331800082202F0FDFD23686E
:108EC000002BF5D0122002F05FFD061E0DD0C1234D
:108ED00021680370457002311022023002F0ECFD6F
:108EE00023683100587802F00FFC206802F01CFC67
:108EF00000232360DCE7C046E065FF1FF8B50400EF
:108F00002020FDF755FB0D4EA700BB590500002B97
:108F10000DD000280BD0D878FF2809D108492A00A5
:108F20000C55F35907480333611802F0C5FCF8BD2E
:108F3000290002F069FB0028F0D1F8E7FC65FF1F6B
:108F4000E465FF1F55A1001170B5064D84006359FB
:108F5000002B05D0D87802F04FFCFF226359DA705D
:108F600070BDC046FC65FF1F70B506008CB00C00DC
:108F7000150000213022684602F056FC3100102214
:108F8000684602F069FB1D2021000322684402F0BC
:108F900063FB6846FFF7D8FD2D210400032228005B
:108FA000694402F059FB20000CB070BDF0B5070019
:108FB000160097B001931CAB1D7830221EAB0091B8
:108FC0000AA800211C7802F02FFC102239000AA800
:108FD00002F042FB1022002102A802F025FC072229
:108FE000310002A802F038FB072202AB9818631E7A
:108FF0009C41019902F030FB02AB9C732B005A1E7E
:10900000934102AAD3730021102206A802F00CFC9F
:1090100006221D9907A802F01FFB1A2002ABC018F8
:1090200006221F9902F018FB102200990EA802F0E8
:1090300013FB102202AB0EA908781C78013A60409D
:10904000D2B2087001330131002AF5D10AA8FFF726
:109050007BFD102212A904000EA802F02DFD1022A3
:1090600006AB0EA908781D78013A6840D2B20870A4
:1090700001330131002AF5D10AA8FFF765FD044349
:1090800010222098E4B212A902F0E6FA200017B0EC
:10909000F0BD70B50E0014008CB0010010226846BF
:1090A0001D0002F0D9FA3100082204A802F0D4FA17
:1090B0002100082206A802F0CFFA6846FFF744FD17
:1090C00004001022280008A902F0C6FA20000CB003
:1090D00070BDF8B506000D0000243719AC4200D36E
:1090E000F8BD02F059FC030A3B70631CDBB2013788
:1090F0009D4203D90234F054E4B2EEE71C00EDE7E0
:1091000073B506000C000225002819D0002917D0DD
:10911000032101A8FFF7DDFF6B469A793F231A4030
:10912000013313436A463000937101A92200FFF70F
:109130001BFF051E04D10322E01C01A902F0BCFCA8
:10914000280076BD03785807DA08C00FD2008000E7
:109150009B0710439B0F1843C0B2704707230B4077
:10916000C908C9000B4303707047000070B50400C4
:10917000FFF7EAFE134DA4006359002B21D0186AB3
:10918000002801D002F0D0FA2B59986E002801D0A7
:1091900002F0CAFA2B59D86E002801D002F0C4FAA6
:1091A0002B59186F002801D002F0BEFA2B59586FC6
:1091B000002801D002F0B8FA285902F0B5FA0023CD
:1091C0002B5170BDFC65FF1F0E4B8000C35870B55E
:1091D0000C00002B0FD09D68002D0CD02B78201D8B
:1091E0000B706B784B70A97CFFF7B8FF2B7E237256
:1091F0006B69E36070BD10220021200002F014FBB7
:10920000F8E7C046FC65FF1F014B18607047C04679
:10921000F865FF1F074A03008000825810B5002A36
:1092200006D0D088984203D1012901D1FFF79EFFD3
:1092300010BDC046FC65FF1FF0B5264E95B08700F7
:109240000B93BB590500099112200A92002B31D0D3
:10925000D888FFF7A5FB04001420002C2AD0280092
:1092600010A9FFF7B1FFBB591E781D6A002E23D04D
:109270000895FDF7EFFA07000020FDF7F1FA0790D7
:10928000A379E61D069310AD0CA9089800F0E2FA48
:109290000EA9280000F0D7FA0B9B0A990493069BAD
:1092A00009980293079B0396019300970EAB0CAAB3
:1092B000FFF77CFE15B0F0BDFDF7CCFA069030004C
:1092C000FDF7CEFAE31DA779079310AB06000893CC
:1092D000DAE7C046FC65FF1F30B50C4C85002A5903
:1092E000030085B00120002A0ED018006946FFF760
:1092F0006BFF2B591A78D888054B002A00D1054BF3
:109300006A46072100F0D9FB05B030BDFC65FF1FA0
:10931000479800115598001130B5094C850029591E
:1093200085B010226846253102F0C6FB2A5911216A
:10933000044BD0886A4600F0C0FB05B030BDC04683
:10934000FC65FF1FF198001130B5094C85002959C3
:1093500085B010226846353102F0AEFB2A59112142
:10936000044BD0886A4600F0A8FB05B030BDC0466B
:10937000FC65FF1F2F990011F7B54D4F8600102097
:10938000F4590D0002F0F8FAF3592062186A13221A
:1093900000286CD0033A29009C6802F08DFBF35939
:1093A0001A780192002A58D11E6A227D317B944698
:1093B00051400122019F114201D167461740217D92
:1093C000914339432175377B4F40BC4660460027A7
:1093D000800701D44F081740012102208F40227DD1
:1093E00082433A432275377B5740BC46604600278C
:1093F000400701D497080F400420227DBF0082431C
:109400003A432275627D002794466046727B424053
:109410000A4201D167460F400121627D8A433A43E7
:109420006275777B5740BC4660460027800701D4B1
:1094300057080F400220627D7F0082431743677503
:10944000767B00227E40760701D4BA080A400426C3
:10945000617D9200B1430A4362756A78002A08D0A0
:109460006278002A05D005220533DA770022100041
:10947000FEBD04222979114205D1A17C114202D1FD
:109480000533033AF1E7019A21782C78002A02D1BA
:109490000A002100140018220429E8D8042CE6D878
:1094A00005206043034A05331218525CDDE7C046CD
:1094B000FC65FF1FD8BE001110B50A001121024B38
:1094C00000F0FBFA10BDC0468B9900110B0030B5BF
:1094D00087B001AD2B806B4604001100981D082257
:1094E00002F0EAFA2A000B212000024B00F0E5FA14
:1094F00007B030BDB399001110B50A001121024B1D
:1095000000F0DBFA10BDC046079A001113B50B003E
:1095100011006A4613706B4604000622581C02F0C4
:10952000CBFA6A4608212000014B00F0C6FA13BDB1
:10953000279A001110B50A001121024B00F0BDFA64
:1095400010BDC046779A00117FB505000B4BAA00ED
:10955000D4580800002C0FD0666F237FE288217852
:109560000396266F0296E66E0196A46E0094FDF7B0
:1095700009FC2800FFF7FAFD7FBDC046FC65FF1F10
:1095800010B51721FFF7E0FF10BD000070B50A000D
:109590000D00064B0221040000F08FFA0600297826
:1095A0002000FFF7D1FF300070BDC0465799001171
:1095B00070B586B000236A461370836804001D7876
:1095C000681E0A2859D801A902F036FA0606333770
:1095D0003B3F43474B4F5300180000F042F906232E
:1095E00012284BD000281BD16088FFF7D9F9082337
:1095F000002813D04279002A47D1264B1A78072336
:1096000012070BD5244B1A680723002A06D01668C8
:10961000002E03D0290001AAB04703006A46137048
:109620006B461B786088002B2AD1FFF767FC06B0D9
:1096300070BD180000F06CF9D4E7180000F087F94D
:10964000D0E7180000F093F9CCE7180000F0ADF96E
:10965000C8E7180000F0C3F9C4E7180000F0F6F9F5
:10966000C0E7180000F0F6F9BCE7180000F013FAA4
:10967000B8E7180000F013FAB4E707236A4613703E
:1096800069466088FFF782FFD1E70523012AC5D12B
:10969000024BB8E78964FF1FF465FF1FF865FF1FE1
:1096A000F8B52C4F8600F35904000D00002B40D074
:1096B000DA8882423DD15A78062A33D11A78002AB4
:1096C0002ED0012099681A6A097D014206D0157BC7
:1096D000054203D007225A700120F8BD0220014242
:1096E00004D0157B054201D00922F4E70420014291
:1096F00004D0127B024201D00B22ECE7164B1B6810
:10970000002BE9D05B68002BE6D020009847BB59BE
:1097100000215B78122BDFD12000FFF715FFDBE77C
:109720000E4BECE7112A04D1002900D03225290084
:10973000F2E7002D08D12000FFF732F9002803D00E
:10974000102302791343037121002800FDF798FAD2
:10975000C2E7C046FC65FF1FF465FF1FF865FF1FE9
:1097600070B50E4E8500AB590400002B13D01B784A
:10977000002B11D10A4B1B68002B04D05B68002B17
:1097800001D02000984773595B78122B03D1002138
:109790002000FFF7D9FE70BD024BECE7FC65FF1F10
:1097A000F865FF1FF465FF1F094B8000C3581020A8
:1097B000002B0CD01A6A002A09D09B68002B06D017
:1097C000127A1B7E101C9A4200D9181CC0B2704736
:1097D000FC65FF1F70B503000D0014000220002A75
:1097E00030D000292ED013700B78081D53704B78A1
:1097F0009370FFF7A7FCE070012002212B7A237100
:109800006B7B034063716A7B0A40134304226371DC
:109810006E7B1640334363716E7BF608F60033436C
:1098200063712B7B0340A371287B014000200B4315
:10983000A371297B0A401343A3712A7BD208D2006B
:109840001343A37170BD10B50A0001000120FFF79A
:10985000C1FF10BD10B50A0001000220FFF7BAFFDA
:1098600010BD70B506000C000220002E30D000297B
:109870002ED07378201D0B70B3784B70F178FFF702
:109880006DFC01223579257271794B100800134067
:10989000934010400343881010408000C9080343E0
:1098A000C9000B436373B1794B1008001340934018
:1098B00010400343881002409200C9081343C900B6
:1098C0000B4321202373FCF773FE854201D2122043
:1098D00070BD2220257AFCF76BFE8542F7D82378ED
:1098E0001820042BF4D86378012BF1D80020EFE77F
:1098F000030010B50220002909D0002B07D0032255
:10990000481C0A7019000D3202F0D6F8002010BD74
:1099100003000222080010B5002B06D0002904D055
:109920000E32591C02F0C8F80022100010BD0300CE
:1099300010B50220002909D0002B07D00422481CB2
:109940000A7019000C3202F0B7F8002010BD10B5F3
:10995000FFF7DEFF10BD03000220002906D0002B18
:1099600004D0052200200A701B784B70704703005A
:109970000220002B08D0002906D05B7800200B7055
:10998000013B082B00D918307047030010B50220A6
:10999000002909D0002B07D00622481C0A701900A4
:1099A0000A3202F089F8002010BD10B5FFF7B0FFB1
:1099B00010BD02000B00022010B500290ED0002AB5
:1099C0000CD007211970118859701188090A9970F3
:1099D00011180822D81C02F06FF8002010BD0300F7
:1099E0000A00022010B5002B0CD000290AD099786B
:1099F0005878090201431180901CD91C082202F0FA
:109A00005BF8002010BD030010B50220002909D02A
:109A1000002B07D00822481C0A701900921802F087
:109A20004BF8002010BD02000B00022010B50029E9
:109A30000BD0002A09D00921197011781818597013
:109A4000511C062202F038F8002010BD10B5FFF7B7
:109A50005FFF10BD02000B00022010B5002A09D0E4
:109A6000002907D05178197011180622581C02F0ED
:109A700023F8002010BD030010B50220002909D0F2
:109A8000002B07D00A22481C0A701900063202F087
:109A900013F8002010BD10B5FFF73AFF10BD02000B
:109AA0000B00022010B5002A06D0002904D01800AF
:109AB0005178FFF753FB002010BDF0B585B01700BB
:109AC0001E006A4606230500080091819380FEF778
:109AD000C0FC1324011E02900CD03800B047041EB5
:109AE00005D1280001A9FEF76FFA041E02D00298E2
:109AF00002F05AF82800FFF701FA200005B0F0BD87
:109B0000F0B504008BB0019115000021102202A8CD
:109B100001F08AFE334EA700B85900283CD0C38814
:109B2000A34239D10378002B36D14278062A18D1C6
:109B300002000100553235310C3006ABFFF7A9FAAF
:109B4000002829D12000FFF72FFE020006A902A855
:109B500001F0B2FF200002A901F05EFD01200BB070
:109B6000F0BD816E002917D00B8A112A28D19D42A1
:109B70000ED101981231093A02F00EF8012807D1EE
:109B8000BB5920009D6EFFF70FFE29000200DEE7A3
:109B900032212000FFF7D8FC2000FEF701FF061E4F
:109BA0001BD0416A002918D00B8AAB4215D108227C
:109BB0000198123101F0F0FF01280ED1716A0AE01C
:109BC0009D42E9D108220198123101F0E5FF0128F8
:109BD000E2D1BB59996E8A7EB9E7200001F0E4FD1D
:109BE000BCE7C046FC65FF1FF0B56B4D87007E5992
:109BF00085B0337802900393002B00D087E0B368E0
:109C0000346A01937078062817D101221B7D134214
:109C100002D0217B114218D10222134202D0217BB3
:109C2000114251D10422134203D0237B134200D0AE
:109C30008BE0019B5A7DEB5991E007380428F8D856
:109C400001F0FAFE032E42678300B36E002B03D1AE
:109C50001C2001F091FEB066EB599C6E002C1CD0CC
:109C600010220021200001F0DFFD0298FFF79CFD8B
:109C700001002000FFF72DFA01F08EFE2082200067
:109C800008211230FFF725FA0298FFF78DFDA07624
:109C9000EB592100D888FFF70FFC0822EB591CE094
:109CA000B36E002B05D01A00198AF0881232FFF724
:109CB0000DFC0222019B197DEB5911423DD0207B06
:109CC00010423AD0073208E0F488FCF7DBFD0100CF
:109CD0002000FFF711FC0A22EB595A70029B9C00EE
:109CE0002A595378073B042B11D8D088FEF758FE29
:109CF00000284ED0C3895A08D2182849029B0298DE
:109D0000CB542B5941180433254801F0D5FD05B03B
:109D1000F0BDFCF79FFD03000120834201D100202C
:109D20000393EB59DE88FCF79BFD0399020030009A
:109D3000FFF7ECFB019AEB59117D042211420CD084
:109D4000217B114209D00B22C7E7F688FCF73CFDC6
:109D500001003000FFF7EEFB6BE7019A527D012115
:109D60000A4204D0607B084201D00C22B5E70221F0
:109D70000A4204D0607B084201D00E22ADE70421E4
:109D80000A4204D0627B0A4201D01022A5E71222C7
:109D9000A3E7FA225200B0E7FC65FF1F0066FF1F31
:109DA0005FA1001110B5064B1A780423100018406B
:109DB0001A4200D00348FFF727FA002010BDC04622
:109DC0008964FF1F4443FF1F70B50400FFF7D4FAF6
:109DD000051E43D12000FFF77FFA234EA400A059AF
:109DE0008268937CDB0708D50321036A1B790B404B
:109DF000012B02D1017F0B430377431DD97F8B1EBB
:109E0000022B0DD8022900D00121C088FCF790FF59
:109E1000042133591A7F59700A431A77280070BDFC
:109E200001290CD102231022437000210C3001F0D3
:109E3000FBFC305910213530FFF74BF9EEE70529CF
:109E4000ECD10223D118437010220C3001F034FE03
:109E500004233259117F0B431377EAE708251828AA
:109E6000DCD1053DDAE7C046FC65FF1FF0B58BB0DD
:109E7000059143887E4F9E00F45915000493002CF1
:109E800015D1012902D000200BB0F0BD101D57786C
:109E90001678FFF757F9EB68320002932B7A049992
:109EA000019300903B002000FCF70CFFEBE7E388F8
:109EB000049A934201D00820E6E72378012B00D1D1
:109EC000D4E0059B581E092800D9CFE001F0B4FD6D
:109ED00005CE0A29CC506C859AB229000498FFF768
:109EE00073FFD1E7200029001022453001F0E4FD86
:109EF000B9594B78042B02D1013B4B70C3E70B00DF
:109F00000A00253335320C310498FFF795F904988F
:109F1000FFF702FA0522431E9841BB59C0005A7050
:109F2000B2E7200029001022553001F0C5FD049B46
:109F30004F4C9D00295904980A0006AB55320C314C
:109F4000FFF77AF929591022453106A801F024FEBD
:109F5000012808D10498FFF7F7F90590002804D1EB
:109F600006222B595A7005988EE708230593FAE7C5
:109F700063780C2B7AD1E36E002B03D11C2001F007
:109F8000FBFCE066BB59D86E00286FD01022290078
:109F900001F092FDBB590498DC6EFFF705FC0D2221
:109FA000A076BB595A706EE7E06E00285ED06378E9
:109FB0000D2B5BD12B8808220382A91C123001F0E3
:109FC0007BFDBB599A68517D0222114226D0186A46
:109FD000407B104222D00C32E4E763780E2B45D14F
:109FE000236F002B03D1162001F0C6FC2067BB595C
:109FF000186F002803D01022290001F05DFD0F2208
:10A00000BB59CFE763780F2B30D1206F0622691C34
:10A01000103001F051FDBB599A68517D0422114264
:10A0200003D0196A497B1142D5D100210498FFF76A
:10A030008BFA28E7636F002B0DD0BB59586F0028AF
:10A04000F3D01022290001F037FD0122BB59524202
:10A050005B6F1A61E9E7142001F08EFCBB59606761
:10A060005B6F002BE9D126E72978DFE707200BE7B4
:10A07000FC65FF1F10B5064C207001F0F5FB0621B2
:10A080002078FDF791FF0348FEF778FC10BDC0462D
:10A090000F66FF1F1592001100200BB270B50D0066
:10A0A000834216DA264B187801F066FB041E0DD0A9
:10A0B0000378922B0ED0A02B37D0224B1878FF2894
:10A0C0003AD0210001F020FB002835D18020000289
:10A0D000684070BD43780E2B0BD03E2BEDD18378BA
:10A0E000052B12D0082BE8D181798088FFF7D8FAA8
:10A0F00008E0154B82889A42DFD183681878591C92
:10A10000FEF7C0FE002817D1D7E7104B1B785B077E
:10A1100012D50F4B1B68002B0ED09B68002B0BD069
:10A12000C289811D80889847ECE7FFF741FAA06853
:10A13000002801D001F038FD200001F075FCC5E7D2
:10A140000F66FF1F3D43FF1F182000008964FF1F9B
:10A15000F865FF1F10B50078FFF712FA10BD10B5B3
:10A160000078FFF7FDFA10BD0C234343084A10B5F1
:10A170009B185A68002A03D0012901D1904710BDCD
:10A180009B68002BFBD00029F9D19847F7E7C04620
:10A190002C66FF1F01238340094A10B5946B1C43B2
:10A1A0009463506B98435063D46B2000984301290B
:10A1B00001D120001843D063116B0B43136310BD12
:10A1C00000800040F0B500240127154B85B0DA6B04
:10A1D000144E03921A6C0192DA64019BE3403B42F5
:10A1E00017D0039DE5403D400295E5B20299280055
:10A1F000FFF7BAFF316A736A002908D03900002BD3
:10A2000001D0029979402800FFF7C4FF01E0002B3C
:10A21000F9D101340C36172CDFD105B0F0BDC046A2
:10A22000008000401066FF1F064B01215A68C240A3
:10A230000A4204D01B68C3401800084070471B6DD9
:10A24000F9E7C046008000400122064B8240002909
:10A2500003D0D9680A43DA607047D9689143D9605E
:10A26000FAE7C0460038004030B5032444430F4BA2
:10A27000E25C1B199C785D7801232D1B0135AB40F6
:10A28000013BA340A140DB430C00122807D808493A
:10A2900092005218116819402143116030BD054ADF
:10A2A00011680B4023431360F8E7C0461FBF00113D
:10A2B00008F0004014F00040C21F70B5D4B206236D
:10A2C000092C0BD80125084C9540002908D0002105
:10A2D000FFF7CAFF23682B4323600023180070BDDB
:10A2E0002368AB43F8E7C04600380040214BF0B587
:10A2F0001B185B78022B21D1032444431E4A1F4EB6
:10A30000A35C12199478012215008540B76B013CBB
:10A31000E4B23D43A240B563194C122815D89B0006
:10A3200000290CD117495B1899680A439A600123E8
:10A33000205C154A834011680B431360F0BD11493E
:10A340005B18996891439960F1E70E4B00290DD194
:10A3500059690A435A61225C1328E8D00123203A44
:10A3600093400A49086803430B60E7E75969914342
:10A370005961F0E71066FF1F1FBF00110080004009
:10A3800064BF001100F00040A0F00040A4F00040C5
:10A39000F8B500241B4E1C4D1C4B1B5D012B1FD11F
:10A3A000194A9269E2401A420BD00122B2569340F8
:10A3B0002200143AD2B2022A09D815494A69134335
:10A3C0004B61013402360C35172CE5D1F8BD002263
:10A3D000B2560F499200521891680B439360F0E710
:10A3E000022BEED1E7B23800FFF71EFF01235840E1
:10A3F000C1B23800FFF77AFF3800FFF715FF687722
:10A40000DFE7C046F1BE00111066FF1F1166FF1F97
:10A4100000F00040012202388240054B002903D0A1
:10A4200059690A435A617047596991435961FAE77A
:10A4300000380040F8B50E0001210F008740114A96
:10A440000400D368FD43BB43D360831E8B4201D815
:10A45000FFF7E0FF00212000FFF72EFF0A4A0B4B19
:10A460005168012E05D139431B1951605E700020DF
:10A47000F8BD2940516002221C1962709A6915408A
:10A480009D61F4E700380040008000401066FF1F27
:10A49000012210B58240074B002906D019680A43F3
:10A4A0001A600121FFF7C6FF10BD196891431960BA
:10A4B000F7E7C046008000400C2370B500254343F9
:10A4C0000A4A29009B181D70094B04001B185D7077
:10A4D000FFF7B0FF0123A340064928000A681A438A
:10A4E0000A6005490A689A430A6070BD2C66FF1F1E
:10A4F0001066FF1F348000403080004070B50400BB
:10A500000E00FF2813D003250540FFF7D5FF084AAA
:10A51000A3089B009B183F22ED00AA40AE4019689B
:10A5200020009143314319600121FFF78DFE70BD7A
:10A5300018380040F8B50C244443134B0500E418C8
:10A540006368002B03D1A3681220002B1AD00222CB
:10A5500001270E4B00215B195A7028002770FFF766
:10A5600069FF63681E1E08D0A3683E00002B04D05C
:10A570002800FFF759FE4640F6B228003100FFF7E9
:10A5800009FE0020F8BDC0462C66FF1F1066FF1FA5
:10A59000F7B5C420FF222B4B8000195800249143AB
:10A5A0003F3A0A431A508022274F5202274E1A6020
:10A5B000274B1D5D002D21D0A31E012B03D80121A7
:10A5C000E0B2FFF727FF012D18D11F4B9B69E34035
:10A5D0002B4213D0E3B218000193FFF725FE0100D0
:10A5E0000198FFF755FFE3B2143B022B1DD8012160
:10A5F0007156184A8D405369AB4353613B7F002B22
:10A600000DD0E5B22800FFF795FF2800FFF70CFEFC
:10A610007B7F0100834202D02800FFF7A5FD0134B3
:10A620000C370236172CC3D1F7BD01210023715618
:10A63000F3568D40074A9B009B189A68AA439A607C
:10A64000DCE7C04600E100E01066FF1FF1BE00112C
:10A650001166FF1F00F0004070B50E0015000400E9
:10A66000FFF72AFF0C236343094A20009B189D60D3
:10A670005E60FFF75FFFF021064B074A8900051E69
:10A680005A5002D02000FFF717FF280070BDC046C7
:10A690002C66FF1F0000FF1FC5A1001170B5134DF0
:10A6A00007202C78002C1FD198222100520028006E
:10A6B00001F0EAF80123C420FF222B700C4B80002C
:10A6C0001C635C630B4B1C605C600B4B1958914323
:10A6D0003F3A0A431A50802252021A600D20074A5C
:10A6E000074901F099F8200070BDC0461066FF1FB1
:10A6F00000800040A0F0004000E100E091A50011C2
:10A7000091A30011030010B50620072B09D8054AB4
:10A71000137001F099F8D7210020034B034A8900F8
:10A720005A5010BD6C43FF1F0000FF1FD91AFF1FB6
:10A7300070B51D0002240C2910D8094ACA40D2075E
:10A740000CD5FBF741FF041E08D1059A0499280097
:10A75000FBF756FFFCF7C4FDFFF724FB200070BD9C
:10A760001210000030B50D7802232C009C431842D3
:10A7700001D02B431C0008252300AB43284201D005
:10A780002B00234320241D00A543204201D01C435D
:10A7900025002A230D70184204D011781E3B0B436C
:10A7A000137030BD0028FCD10C2113788B43F7E7E0
:10A7B000F8B51D0006AB1B88140007AA0E000B207D
:10A7C0001778002B27D10A78022A49D14A68507895
:10A7D00011780002244A08438018042840D801F068
:10A7E0002BF903121D1B2300F06801F045F9021C30
:10A7F000C0B2B84200D93A1CD2B22000F1682A8017
:10A8000001F05AF906E00222F3681B882A802370BF
:10A810001B0A63700020F8BD0622EEE701232B809F
:10A82000F3681B782370F5E7F368002B16D0082235
:10A830002A801A8822701A88120A62705A88A270B6
:10A840005A88120AE2709A8822719A88120A6271F2
:10A85000DA88A271DB881B0AE371DBE72B80D9E77A
:10A8600001202B80D7E7C04600D6FFFFF7B51600C2
:10A870000A781D0008AB1F880C000123022A18D19A
:10A880004A685078117800022B4A08438018032840
:10A890000FD801F0D1F802254439E06801F0ECF856
:10A8A000C0B20723B84204D37B190193152B02DDF4
:10A8B0000D231800FEBDE0682A003100C01901F028
:10A8C000FBF86B4600209B88E268D0541B4B1B684A
:10A8D000834203D01B68834200D098470023E8E7F7
:10A8E0000B23002FE5D1022DE2D1737832781B02C1
:10A8F0001343E2681380114B1B68002BEED01B68DA
:10A90000002BEBD00120E8E70B23002FD1D1062D3F
:10A91000CED12A003100E06801F0CEF8DEE70B234B
:10A92000002FC6D1012DC3D132787533012AC0D88A
:10A93000E3681A70D2E7C04600D6FFFF1C68FF1F0D
:10A9400070B50C001500072837D801F075F804140D
:10A9500036361B36242E182015290BD8184E1622F1
:10A960000021300000F060FF22002900300001F0DB
:10A97000A3F8002070BD18200229FBD11288114BCA
:10A980001A80F6E718200829F4D10A000E48290099
:10A9900001F0BAF8EDE718200129EBD10B4B107844
:10A9A0000B49DA69FFF7DEFEE3E718200129E1D160
:10A9B000064B10780749DA6BF4E70220DAE7C04665
:10A9C0000468FF1FEA43FF1FE043FF1F7043FF1FA0
:10A9D0009843FF1FB843FF1F030010B50020DB079B
:10A9E00004D50721024A034800F08CF810BDC04688
:10A9F0007CBF00117043FF1F054A03001068002848
:10AA000003D082889A4201D1806870470068F6E7D7
:10AA1000146AFF1F0A88030008009A4204D08A883B
:10AA200004309A4200D0002070470000F8B5F222AE
:10AA300000230D4F0D4E7968050042433370994253
:10AA400000D07B600A4C0021200000F0EDFE0023C6
:10AA50001A007C60AB4202D100203370F8BD013394
:10AA60002280DBB2F234F5E70C6BFF1F0A6BFF1F8D
:10AA7000186AFF1F73B56B46019006006846150003
:10AA80001980FCF75FFF041E11D1002D0FD07689CD
:10AA9000002E11D00C2000F06FFF00280ED0084AC5
:10AAA0000460136886808560002B02D1106020004E
:10AAB00076BD1A001B68F7E70224F8E71324F6E7CF
:10AAC000146AFF1F012100220A4B10B549420A4CAB
:10AAD000198099809A719A70084B20700120198012
:10AAE0005A60FFF7A3FF2078FCF78AFF0448FDF7C0
:10AAF00045FF10BD2468FF1F146BFF1F0C6BFF1F69
:10AB0000B1AB0011022310B5002802D0FFF7B2FF4D
:10AB10000300180010BD0000030010B50020DB0783
:10AB200004D50421024A0348FFF7A4FF10BDC04624
:10AB300090BF0011F043FF1FF0B50E2687B00393BE
:10AB40000CAB1F8802ABF61805000800310002921A
:10AB5000FDF77AF804000120002C0FD03088FFF7B1
:10AB60004BFF03000E20002B08D05E68002E05D09E
:10AB700021002800039B029A0097B04707B0F0BD60
:10AB80000A4B10B5984207D10122002352420A8095
:10AB90008B708A808B7110BDFFF73CFF0028FAD0C4
:10ABA00001235B42038000238370F4E7FFFF000072
:10ABB000F8B5050001290AD1134E00243388F22785
:10ABC000AB4219D028001149FFF7DAFF06E002294D
:10ABD00004D10139FDF750FF0028EDD0F8BD3B004E
:10ABE00063437268D018D35A002B09D03A00002171
:10ABF00000F01AFE0134E4B2054B1B78A342EED8F4
:10AC000001235B423380DDE70C6BFF1F2468FF1FCD
:10AC10000A6BFF1F10B5FFF7FDFE03000020834203
:10AC200000D0987810BD0000F0B589B01C000EABC4
:10AC300080CB03901E8810AB1B78049202930B7A92
:10AC40000D00DB0616D42B780593022B24D0049834
:10AC5000FFF7D2FE002812D003689C46002B0ED0CE
:10AC6000029B2200019329003B0064460398009652
:10AC7000A04705E00498FFF7BFFE002802D10E2090
:10AC800009B0F0BD8368002BF9D00A22290003988F
:10AC900098470028D7D0F3E76B6858781A786B4B41
:10ACA000000210439842D2D8043B984210D2684B1D
:10ACB000984242D015D8674BC0180128C7D80B203E
:10ACC000002EDDD1EB681A7859683A80200028E020
:10ACD000614BC018032800D979E000F0ADFE846A0A
:10ACE000789E5E4B9842B2D10B20002EC8D1012332
:10ACF0003B80EB6831001B7823706889013080B29B
:10AD0000FCF7A2FF3A88031E0ED0017802328A189F
:10AD10003A80428962704289120AA27059680278A8
:10AD2000E01C00F0C9FE06E004323A803100042243
:10AD3000601C00F079FD0020A2E70B20002E9FD1BF
:10AD4000EB6807A91E8804233B80330A3000267075
:10AD50006370FCF779FF051E28D004AB9A890E2397
:10AD600004A95B183E49C668FCF7E2FF00280BD136
:10AD70002B783C486A680599FBF798FB002803D1BB
:10AD8000012304AA5B42D3813278022A06D171687A
:10AD9000201D00F091FE3B8802333B800E2304AA65
:10ADA0009B181B88A3701B0AE370C4E704ABDE8109
:10ADB000F4E70B20002E00D062E7E9680398FFF764
:10ADC00029FF02233B802070000A6070B3E70B204C
:10ADD000002E00D054E70222EB681B883A802370D3
:10ADE0001B0A6370A7E7E86800F046FEC2B20300E2
:10ADF0000720B24200D243E70DD00299DBB27118AE
:10AE0000994202DB921BD3B20293029BE9681A00BB
:10AE10003B8089195AE70023F6E70B20002E00D06B
:10AE20002EE70722EB683A801A7822705A7862700F
:10AE30005A88A2705A88120AE2701A792271DA8846
:10AE40006271DB881B0AA37175E7C0460429000004
:10AE50000228000000D8FFFFFFD6FFFF03280000F4
:10AE6000FFFF0000C0BE0011F0B58DB06B460020A2
:10AE7000089120229B5E83423DDAA64B187800F0B1
:10AE80007BFC071E32D00378B02B2CD1007902381E
:10AE900016281FD800F058FE17001E001E001E00C6
:10AEA00031001E0096001E001D011E0052011E00F2
:10AEB00073011E00CD011E0050021E001E001E0068
:10AEC0008E021E00E302944B94491B8878880B8005
:10AED000FBF72CF83800FCF7ADFF914B1B68002BFB
:10AEE00001D038009847380000F09EFD8020089B74
:10AEF0000002434018000DB0F0BDEE22002187484B
:10AF000000F092FC0BAA3B7B7989388900923A00C9
:10AF10000D32FCF7B1FD0400804B1B78002C3FD1B3
:10AF200046E0804B788805937F4B4100CB5A0BAEAF
:10AF3000073BDBB232880293002301937B4B210055
:10AF400006930093059BFFF76FFE744D002810D108
:10AF5000069B3A8A1B889A420BD138000599123019
:10AF600000F01AFE002804D02B7862899B00EB18B1
:10AF70005A80162306A81B18328820007989FCF70E
:10AF8000D7FE2B7804009A00AA1851880029C3D054
:10AF90000133DBB22B70002807D006A9C98A918043
:10AFA000634A12889A42BCD802E00121494291804A
:10AFB000002B04D059497888FAF7ECFF8AE73E89DC
:10AFC0000A2479E000253E89574B06937B88069A30
:10AFD0005B009B5A033B9D4202DB002DF0D05BE0FF
:10AFE000162206A812183B7B798900923A0030009D
:10AFF0000D32FCF741FD0590002858D04689017AB2
:10B000007888FCF703FD041E44D1464B78880793EB
:10B01000069B4100C95A454B0439C9B206AAD28AD7
:10B0200006930291019400930599079BFFF7FCFD9D
:10B03000041E2FD1069B39491A88931C002D26D156
:10B040004B807988384B4900CB5A5119033B8B42CE
:10B0500020DD059B31485B8941190B71A91C013525
:10B06000C9B2EDB2059145191B0A2B71059B2D49FB
:10B070000433181800F020FD2C4B059A1B88D318B8
:10B08000DDB22C4B9E4205D00136B6B29CE7498812
:10B090009942D6D0002D0CD0204C2800618800F0B9
:10B0A0008BFB207021007888FAF784FF12E7059C5B
:10B0B000F0E7002C00D183E77B78142B00D109E75F
:10B0C00016493B794E800B700C717888FAF724FF93
:10B0D00000E7162406ABE41821003889FCF7B4FD1C
:10B0E000011E00D1B7E1788822880F4C45002C5B07
:10B0F0000A4D013CE4B2029400240F4B01940095E8
:10B10000FFF792FD041E00D014E129007888FAF7B9
:10B1100061FFDFE6146BFF1FDC42FF1F2C68FF1F7F
:10B120002068FF1F2069FF1F5C64FF1F106AFF1F5C
:10B13000DA42FF1FFFFF00002E68FF1F162406AB38
:10B14000E41821003889FCF77FFD011E00D182E15F
:10B1500078882288AE4C45002C5BAE4D013CE4B2B1
:10B1600002947C89AC4B01940095FFF75DFD041EB1
:10B1700000D0DFE029007888FAF736FFAAE600253C
:10B18000A44B1D803B00F6331B78A24A78880792B7
:10B19000AB4208D99E4B12880693069943005B5A2E
:10B1A000013B9A4203DB0799FAF728FF92E616243F
:10B1B0006B00FB18059306ABE418059B210018896A
:10B1C000FCF742FD011E03D1059B01241E8973E794
:10B1D0007888924B2288069C099343001B5B904E13
:10B1E000013BDBB20293002300960193099BFFF71A
:10B1F0001BFD041E02D0059B1E895DE77B88069A15
:10B200005B009B5A079A108832881218934202DC1E
:10B210001B1A013B33807F4C023032880999001998
:10B2200000F04AFC2388328801359B182380EDB258
:10B23000A8E70BAA3B7B7989388900923A000D3246
:10B24000FCF71AFC00250590059B002B04D10A246D
:10B25000002D00D16EE060E0059B7888197AFCF73C
:10B26000D5FB0100041E63D1694C6C4B78880694B1
:10B270000993069B4400E45A694B063CE4B20BAECA
:10B28000328807930294019100930599099BFFF777
:10B29000CBFC041E4CD1079B5E491B881A1D002D58
:10B2A00030D14A80059B5B4C5A8963191A716B1C1B
:10B2B0009BB2E318120A1A71162306A832881B18CB
:10B2C00079890598FCF734FDFF21AA1C2E1D033552
:10B2D0000B00059092B2B6B2ADB2002803D006AB17
:10B2E000DB8AD9B21B0AA218651911712B714C4D5A
:10B2F000301D2A884949201800F0DEFB2B88F618FB
:10B30000B5B2A1E74988914207D17A8806995200DF
:10B31000525AEB18053A9A42C4DC3E4C2800618828
:10B3200000F0FAFB207021007888FAF771FED1E571
:10B33000002DF2D13E89BFE6162606ABF618310085
:10B340003889FCF781FC3D000400FA3500282DD037
:10B35000037A9B060CD400227B8939897888009275
:10B360003A000C32FFF7E8FB041E10D03E8915E0CE
:10B370003088FFF741FB00281AD08368002B17D0D4
:10B380002100122278889847041EE4D0EEE72B783B
:10B39000002B02D17888FAF74BFE00262B78002B81
:10B3A00000D097E5002C00D194E585E60124DDE787
:10B3B0000E24DBE7162506ABED1829003889FCF7CB
:10B3C00043FC041E47D0037A9B0611D4154A7B88A0
:10B3D0001188994203D01448814207D11380134B3E
:10B3E000F2261D780023D9B2A94221D30924A1E76E
:10B3F0002888FFF701FB00282FD08368002B2CD072
:10B400002100122278889847041EDFD092E7C046B8
:10B410005C64FF1F2C68FF1F2E68FF1F2069FF1F41
:10B42000106AFF1F0C6BFF1FFFFF00000A6BFF1F5E
:10B4300031005943546801336018615A0029D2D150
:10B440003C0008342100F22200F036FB210078880D
:10B45000FAF7F6FD3EE501246CE70E246AE71D4B82
:10B460001A887B889A4231D07888FAF7F3FD31E563
:10B47000F223059851684343CD18C95A00291FD0BB
:10B480003B7A012B0BD16C88AB887888AA1D00947D
:10B49000FFF752FB041E02D000233B722E88F222DB
:10B4A0000021280000F0C0F900232B80059B013308
:10B4B000DBB20593084B05991B78064A8B42D7D817
:10B4C00001235B421380002CCED0F5E5002634002A
:10B4D0000596EFE70C6BFF1F0A6BFF1F70B50400AA
:10B4E0000E001500FFF796FA031E08D1310005483B
:10B4F000FFF790FA03001120002B02D01C800020DF
:10B500009D7070BDFFFF0000F8B50B4F06003B7843
:10B510000D001400FF2B0ED00A2000F035FA011E9A
:10B5200009D0B1230380002346800371C5800481C4
:10B53000387800F0E9F8F8BD3144FF1FF7B50F0087
:10B5400008A90600088809A90B240988002821D128
:10B550000234022B1ED1557813782D021D432B0087
:10B560008B4301937334002B14D1FB683000190016
:10B570000093FFF74FFB019C85420BD02A0030005F
:10B580000099FFF7ABFF041E04D12A00300079892F
:10B59000FFF7BAFF2000FEBDF0B50E7885B003902E
:10B5A0000AA805880120022E0DD14C6827786478FE
:10B5B00024023C43054FBC4205D10398DBB20196FF
:10B5C0000095FFF7BBFF05B0F0BDC04602290000A3
:10B5D000034B10B51B68002B00D09847FEE7C04610
:10B5E000186BFF1F07B501A8FFF7F2FF044A0548D3
:10B5F0000021121A00F048F9F8F7FCF8FEE7C046FF
:10B600001C6BFF1F3444FF1F01B40248844601BC79
:10B61000604700BF5147010001B40248844601BCA5
:10B62000604700BF311B000001B40248844601BCE2
:10B63000604700BF193BFF1F01B40248844601BCAC
:10B64000604700BF193AFF1F01B40248844601BC9D
:10B65000604700BFC51D000001B40248844601BC1C
:10B66000604700BF4551010001B40248844601BC57
:10B67000604700BF1D4B010001B40248844601BC75
:10B68000604700BF8538FF1F01B40248844601BCF3
:10B69000604700BF456B010001B40248844601BC0D
:10B6A000604700BF350E000001B40248844601BC6B
:10B6B000604700BFC52DFF1F01B40248844601BC8E
:10B6C000604700BF090E000001B40248844601BC77
:10B6D000604700BF7918000001B40248844601BCED
:10B6E000604700BF792DFF1F01B40248844601BCAA
:10B6F000604700BF691F000001B40248844601BCD6
:10B70000604700BF5549010001B40248844601BCAE
:10B71000604700BF594F010001B40248844601BC94
:10B72000604700BFC521000001B40248844601BC47
:10B73000604700BF014C010001B40248844601BCCF
:10B74000604700BF6571010001B40248844601BC36
:10B75000604700BF6DBC000001B40248844601BCD4
:10B76000604700BF8D12000001B40248844601BC4E
:10B77000604700BF0132FF1F01B40248844601BC8C
:10B78000604700BFF54E010001B40248844601BC89
:10B79000604700BFD92FFF1F01B40248844601BC97
:10B7A000604700BFC94A010001B40248844601BC99
:10B7B000604700BF091B000001B40248844601BC79
:10B7C000604700BF350E000001B40248844601BC4A
:10B7D000604700BF4D38FF1F01B40248844601BCDA
:10B7E000604700BF5D17000001B40248844601BCF9
:10B7F000604700BFA54F010001B40248844601BC68
:10B80000604700BF1147010001B40248844601BCF3
:10B81000604700BF5952010001B40248844601BC90
:10B82000604700BF6130FF1F01B40248844601BC7D
:10B83000604700BF154D010001B40248844601BCB9
:10B84000604700BFC9A9000001B40248844601BC9A
:10B85000604700BFD91AFF1F01B40248844601BCEB
:10B86000604700BF4537FF1F01B40248844601BC52
:10B87000604700BFC926000001B40248844601BCED
:10B88000604700BFC538FF1F01B40248844601BCB1
:10B89000604700BFB70E000001B40248844601BCF7
:10B8A000604700BF1930FF1F01B40248844601BC45
:10B8B000604700BF055E000001B40248844601BC39
:10B8C000604700BFA946010001B40248844601BC9C
:10B8D000604700BF75A9000001B40248844601BC5E
:10B8E000604700BF2526000001B40248844601BC21
:10B8F000604700BFD91B000001B40248844601BC68
:10B90000604700BF2146010001B40248844601BCE3
:10B91000604700BF5933FF1F01B40248844601BC91
:10B92000604700BF9135FF1F01B40248844601BC47
:10B93000604700BFC56D010001B40248844601BCE8
:10B94000604700BFADAE000001B40248844601BCB0
:10B95000604700BF3D18000001B40248844601BCA6
:10B96000604700BFB14E000001B40248844601BCEC
:10B97000604700BFE117000001B40248844601BCE3
:10B98000604700BF3D4B010001B40248844601BC42
:10B99000604700BF1D4D010001B40248844601BC50
:10B9A000604700BF2951010001B40248844601BC30
:10B9B000604700BF9D35FF1F01B40248844601BCAB
:10B9C000604700BFE548000001B40248844601BC5E
:10B9D000604700BF7139FF1F01B40248844601BCB3
:10B9E000604700BFB54C010001B40248844601BC69
:10B9F000604700BFE928000001B40248844601BC4A
:10BA0000604700BFED4A010001B40248844601BC12
:10BA1000604700BFF94C010001B40248844601BCF4
:10BA2000604700BF5125000001B40248844601BCB4
:10BA3000604700BF434D010001B40248844601BC89
:10BA4000604700BF2D3BFF1F01B40248844601BC84
:10BA5000604700BFF30E000001B40248844601BCF9
:10BA6000604700BF2932FF1F01B40248844601BC71
:10BA7000604700BF0D52010001B40248844601BC7A
:10BA8000604700BFDD52010001B40248844601BC9A
:10BA9000604700BF5118FF1F01B40248844601BC33
:10BAA000604700BF851F000001B40248844601BC06
:10BAB000604700BF4D1F000001B40248844601BC2E
:10BAC000604700BFE94C010001B40248844601BC54
:10BAD000604700BF8552010001B40248844601BCA2
:10BAE000604700BF4550000001B40248844601BCD5
:10BAF000604700BF7D18FF1F01B40248844601BCA7
:10BB0000604700BF291C000001B40248844601BC04
:10BB1000604700BF810E000001B40248844601BCAA
:10BB2000604700BF090E000001B40248844601BC12
:10BB3000604700BFC12FFF1F01B40248844601BC0B
:10BB4000604700BF9DA9000001B40248844601BCC3
:10BB5000604700BF413BFF1F01B40248844601BC5F
:10BB6000604700BFB352010001B40248844601BCE3
:10BB7000604700BF0124000001B40248844601BCB4
:10BB8000604700BFEDA5000001B40248844601BC37
:10BB9000604700BF156B010001B40248844601BC38
:10BBA000604700BFCD4C010001B40248844601BC8F
:10BBB000604700BFD949010001B40248844601BC76
:10BBC000604700BF2124000001B40248844601BC44
:10BBD000604700BF3555000001B40248844601BCEF
:10BBE000604700BFDD66010001B40248844601BC25
:10BBF000604700BF8B52010001B40248844601BC7B
:10BC0000604700BFED39FF1F01B40248844601BC04
:10BC1000604700BF9136FF1F01B40248844601BC53
:10BC2000604700BFC135FF1F01B40248844601BC14
:10BC3000604700BF5522000001B40248844601BCA1
:10BC4000604700BF0539FF1F01B40248844601BCAC
:10BC5000604700BF3938FF1F01B40248844601BC69
:10BC6000604700BF017F000001B40248844601BC68
:08BC7000604700BF056A0000F7
:10BC78000003010302020303040205000602070091
:10BC8800080009020A030B030C000D000E030F0342
:10BC9800100311031300140015031603C93B001108
:10BCA800FD3B00110000000002000000BABC0011BA
:10BCB800192A0F180A000000F1590000FD2400009D
:10BCC800414601008580001199A00011ED74001112
:10BCD800897E0011FD52001169AE0011654F0011F7
:10BCE800BD3D0011ED3E00110000000016160000D9
:10BCF8000200000004BD0011F4FFF3FFD2FC0000B5
:10BD08002D4000110000000000000000547579610A
:10BD18000042312E3400303031380067697468755C
:10BD2800622E636F6D2F70767678005448303544F4
:10BD3800000000000200000050BD0011292A282A36
:10BD4800272A262A252A242A0A180000E2040000A5
:10BD58007102000078EC0000744000001027000019
:10BD680060F0000006640000204E000000000000A3
:10BD7800050000001F501D00023CB400000118001F
:10BD880014000000A1020000303132333435363758
:10BD9800383941424344454600000000015700112C
:10BDA800555700110000000002000000BCBD001142
:10BDB8006F2A6E2A1A18EAD8BC80F0FC60000000CE
:10BDC8000000000000005F066B2F363D7D077F3FB7
:10BDD800777C596E7971AF066D4FC6CBEB0EEFCFFE
:10BDE800EEC3A966E9E8FA60D6F46CBCBEE0FEFCD6
:10BDF800EE3E9A769E8E000001A000000000000032
:10BE08006410B71DC8206E3BAC30D9269041DC7653
:10BE1800F4516B6B5861B24D3C7105502083B8EDFD
:10BE280044930FF0E8A3D6D68CB361CBB0C2649B21
:10BE3800D4D2D38678E20AA01CF2BDBDFB349B5F46
:10BE4800800000800010000000000000EF6000117A
:10BE58007977001113610011817B0011976100113E
:10BE6800577B00110D6200112D7B00115F620011DC
:10BE7800F57C0011C7620011F57C0011F962001110
:10BE8800AF7C00110D620011E57A00118562001186
:10BE98008D7C001100000000000000006B630011A1
:10BEA8008D7C0011CD63001191770011052A042AB9
:10BEB800012A002A0229032801280028011800184D
:10BEC80000000000000000000000000000000087E3
:10BED800010102010201010201020303040103013D
:10BEE800010101010303020103000D000E0010000F
:10BEF800110013001401070108010A010B011C01BC
:10BF08001D02040205020702080219021A021C0295
:10BF18001D030103020317000201000504000807BE
:10BF2800000B0A001716001D1C010201010504017F
:10BF38000E0D011110011413011716011A1902022E
:10BF480001020B0A020E0D02111002141302171639
:10BF5800030504030807030B0A030E0D000102037F
:10BF680007090A0B0E0F101112141718191A1B1FA4
:10BF780020212200B1A700116DA8001100000000C7
:10BF880002000000C6BE00110000000099B50011B3
:0CBF98000000000002000000C4BE001108
:020000041FFFDC
:1000000000000000253D0011C0BC0011BCBC001167
:100010004061FF1F00000000000000000000000021
:1000200000000000000000000000000000000000D0
:1000300000000000000000000000000000000000C0
:1000400000000000000000000000000000000000B0
:1000500000000000000000000000000000000000A0
:100060000000000000000000000000000000000090
:100070000000000000000000000000000000000080
:100080000000000000000000000000000000000070
:100090000000000000000000000000000000000060
:1000A0000000000000000000000000000000000050
:1000B0000000000000000000000000000000000040
:1000C0000000000000000000000000000000000030
:1000D0000000000000000000000000000000000020
:1000E0000000000000000000000000000000000010
:1000F0000000000000000000000000000000000000
:1001000000000000000000000000000000000000EF
:1001100000000000000000000000000000000000DF
:1001200000000000000000000000000000000000CF
:1001300000000000000000000000000000000000BF
:1001400000000000000000000000000000000000AF
:10015000000000000000000000000000000000009F
:10016000000000000000000000000000000000008F
:10017000000000000000000000000000000000007F
:10018000000000000000000000000000000000006F
:100190004D32FF1FAD30FF1FC1660100000000009F
:1001A000000000000000000000000000000000004F
:1001B000000000000000000000000000000000003F
:1001C000000000000000000000000000000000002F
:1001D000000000000000000000000000000000001F
:1001E000000000000000000000000000000000000F
:1001F00000000000000000000000000000000000FF
:1002000000000000000000000000000000000000EE
:1002100000000000000000000000000000000000DE
:1002200000000000000000000000000000000000CE
:1002300000000000000000000000000000000000BE
:1002400000000000000000000000000000000000AE
:10025000000000000000000000000000000000009E
:10026000000000000000000000000000000000008E
:10027000000000000000000000000000000000007E
:10028000000000000000000000000000000000006E
:10029000000000000000000000000000000000005E
:1002A000000000000000000000000000000000004E
:1002B000000000000000000000000000000000003E
:1002C000000000000000000000000000000000002E
:1002D000000000000000000000000000000000001E
:1002E000000000000000000000000000000000000E
:1002F00000000000000000000000000000000000FE
:1003000000000000000000000000000000000000ED
:1003100000000000000000000000000000000000DD
:1003200000000000000000000000000000000000CD
:1003300000000000000000000000000000000000BD
:1003400000000000000000000000000000000000AD
:10035000000000000000000000000000000000009D
:10036000000000000000000000000000000000008D
:10037000E5B50011000000000000000000000000D2
:10038000000000000000000000000000000000006D
:10039000000000000000000000000000000000005D
:1003A000000000000000000000000000591AFF1FBC
:1003B000000000000000000000000000000000003D
:1003C000000000000000000000000000000000002D
:1003D000000000000000000000000000000000001D
:1003E000000000000000000000000000000000000D
:1003F00000000000000000000000000000000000FD
:08183800206FFF1F4118FF1F84
:10184000024981F3088802F06FFA0000206FFF1F41
:1018500010B502F089FA072804D0122808D002280F
:1018600008D010BD044A0420136B01331363F8E75A
:101870000220F6E71420F4E70465FF1FF8B507001F
:101880000C0026002500503630785135002804D150
:101890000300287058342370F8BD2978CA00481E08
:1018A0008141A3183800A25C5B68C9B2FFF7D0FF82
:1018B00000280DD12B78DA00A218013350602B706C
:1018C0003378044A013B3370136A01331362D8E75B
:1018D0000123DFE70465FF1F5C234343074910B57D
:1018E000C9180B0058331B78012B05D1FFF7C6FF31
:1018F000034A936A0133936210BDC0463865FF1FE7
:101900000465FF1F10B502F037FB064A01211300E2
:1019100010CB4942D967044B136002F0E5F920006F
:1019200010BDC04600E100E01000100010B504003A
:1019300002F022FB024B1C6002F0D6F910BDC0463B
:1019400000E100E0431E5A425341A022F0B5D2010B
:101950005B421340154D164A40019B182A18127E0F
:101960008BB00191002A1BD01A000832D46F0022DC
:10197000E6B206AFE4B294420EDC2818C369002B2D
:1019800008D0019902AA117106AA049202AA16733C
:1019900003A898470BB0F0BD1978B9540132EAE7B3
:1019A0001A7D1A7806AB01261A70E6E7C467FF1F96
:1019B00000400040F0B5254B04004001C25C85B0FA
:1019C000002A2BD01A18117E002927D0917E0029D9
:1019D00024D01179022921D11689D788D168F51B25
:1019E000ADB22A1C102D00D9102292B2BE4217D1DE
:1019F0001818012303710023C269C38003819A422E
:101A000006D06846032103730171029301A8904731
:101A10000820002C00D0192001F0FEFA05B0F0BD1E
:101A2000013C65426C41A0256442ED012C40084D0B
:101A30001B186419074D0633013A92B2AA42EDD041
:101A40001888461C1E80085C2070F5E7C467FF1FDD
:101A500000400040FFFF00000F220E4B10B59868B9
:101A6000104002380A280BD802F060F80D0A0B0A61
:101A70000A110A0A0A0A060002210020FFF762FF83
:101A800010BD0121F9E70020FFF794FFF8E7DB6FB5
:101A9000F6E7C046004000400F220E4B10B5986894
:101AA000104002380A280BD802F040F80E0A0B0A40
:101AB0000A120A0A0A0A060002210120FFF742FF61
:101AC00010BD01210800F9E70120FFF773FFF7E7D8
:101AD000DB6FF5E70090004013B5334C2378072BFC
:101AE0003DD8324B1A78324B002A39D180221968FE
:101AF00052020A431A60252001F0C4FE20232D4A19
:101B000011680B43802113606B460422C9050868E5
:101B10000733104228D080210422C905C86810422A
:101B20002ED080212020C905CA688243CA601422B1
:101B30001A701A78002A2FD18021C905C86820326E
:101B40000243CA6014221A701A78002A28D11A4B4C
:101B50001A7D22785A601D221A705932DA6013BD3C
:101B60001A6816490A40C5E7086802430A60142249
:101B70001A701A78002ACED01A78013AD2B2F7E752
:101B8000C8680243CA6014221A7019784A1ED2B279
:101B90001A700029F9D1C4E71A78013AD2B2C7E71E
:101BA0001A78013AD2B2CEE76C43FF1F3444FF1FCC
:101BB0003CF000406443FF1F00200040FFFFFEFF99
:101BC000564B70B51B68012B03D1554A936D0133F9
:101BD000936502F011F9534B534A1860534B544C20
:101BE0001A600123534A1360534A13602378002B71
:101BF00006D006225149524802F0A6F8002323706D
:101C0000504A514B10681B78C1B2002B0ED14F4C7B
:101C1000C0B223785BB2002B4FDB237824785BB211
:101C200064B21B0424021B191B1813600B1C5029DF
:101C30004ED95023464A47491078DBB2FF2202288A
:101C40004BD10868444C454D267890432A789642FB
:101C500054D9227824782E78023B5D10A31B6B4365
:101C60005201D31A10335B111843086002F054F983
:101C7000031F012B45D83A4B1B78002B06D0394B5C
:101C80001B78002B02D0002002F05EF9A122364B17
:101C900092009978354B4A431B689B188322920027
:101CA0009B181B78033B012B03D8AF20400001F0A9
:101CB00093FF01222E4BDA8270BD237824785BB229
:101CC00064B2FF33FF341B0424021B190138ABE755
:101CD000CAB2022AAED20223ACE70868254C264DD0
:101CE000267890432A78964208D9227824782D784D
:101CF000023B5B10641B63435201B2E72378DBB203
:101D0000B2E70228D5D11D4B1B78013B022B03D92A
:101D10001B4B1B78022BCCD16C20C8E79809FF1F06
:101D2000FC0FFF1F3C64FF1FFF3F00001410034027
:101D30004064FF1F0C10034000100340D50BFF1F31
:101D40007211FF1FB40003408C09FF1F680AFF1FB8
:101D5000490AFF1F94000340460AFF1F470AFF1F5E
:101D6000F908FF1F2209FF1F300DFF1F3409FF1F55
:101D7000BC0BFF1F440AFF1F450AFF1F1C09FF1F62
:101D80002309FF1F10B502F0B7F80022014B1A809B
:101D900010BDC0463A64FF1F10B502F055F8A121EE
:101DA000054A89009478054A61431268044B521829
:101DB000528C1A8010BDC046300DFF1F3409FF1F22
:101DC0003A64FF1F10B50D4B0D4A9978A1239B0073
:101DD0004B431268D218531DD97F0A4B1B88994276
:101DE00009D2441C07D0C82805D0D2695B1A5A43CF
:101DF000054B5343C01801F0E7FF10BD300DFF1F26
:101E00003409FF1F3A64FF1F7102000070B5244DB2
:101E10002B68002B28D001F017FF2B68D8402B68C7
:101E20000400002B27D002F0B7F82B68D8401D4BD8
:101E30001D4A9978A1239B004B431268D118D25CAC
:101E400091239B00002A20D0CA580132CA50174B58
:101E500017491B680868834214D3D23B181A012A19
:101E60001AD0144B186070BD01F0EEFE124B1968C9
:101E700001F082FED3E702F08FF80F4B196801F0F2
:101E80007BFED4E70D495B18E8E7CA500C4B1B6892
:101E9000DB68E418201AE4E7F530FF30E1E7C046DC
:101EA0001C08FF1F300DFF1F3409FF1F9C09FF1F77
:101EB0003C64FF1FA009FF1F1808FF1F2DFF3F00F4
:101EC0004464FF1F70B504000D00282916D10300DB
:101ED000A433C2881B889B1A0B4A9BB293420DD92C
:101EE00006006A3605223100653001F0F5FF002852
:101EF00004D13100200002F01FF870BD290020003D
:101F000001F00AFFF9E7C046FE7F0000F8B50500C2
:101F1000012001F0B1FF134CA36AA26A9342FBD1E6
:101F2000114E336001F038FE10490300086010487C
:101F3000426894460F4A17680022BC4501D24268A5
:101F4000BA1A0D4802603268AD18A422E562606AD0
:101F5000520302436262094A1278002A01D00F3B01
:101F60000B60F8BD00F00040340AFF1FE408FF1FBB
:101F700028100040180AFF1F1C0AFF1F1C09FF1F22
:101F800070B580241025E405A3682B43A36001F0FD
:101F90000BFEA368AB43A36070BD0000F7B516004D
:101FA00080221C001023D2050191916805000B438B
:101FB000936000225A4BD7301A6001F055FE9D23E2
:101FC0002A002F009B00EB58CA3201210092FC37F7
:101FD000002B01D00021009A386801F0D5FE2900BD
:101FE000009BCB311A784F4BD3351A604B780A7867
:101FF0001B0213438A7812041A43CB781B0613433F
:10200000494A1BBA13604B790A791B0213438A7938
:1020100012041A43CB7931001B061343434A1BBAFF
:1020200013606B782A781B021343AA7812041A43B0
:10203000EB781B0613433E4A1BBA1360019A330226
:1020400013433C4A13603C4B22001B1B9C46032954
:102050003DDCB3089A0013005142B21A032A46D15C
:10206000354AE018511A827840781204000202437F
:10207000E05C043302430A600022FF2B4BDDF022B8
:102080002E4B12011A600F222D4B1A602D4A136835
:10209000002BFCD00023224A27491360091B321D64
:1020A0000B191B68043A180A23706070180C1B0E79
:1020B000A070E3700434002AF2DC802210213B6817
:1020C000D20501333B6093688B439360F7BD634651
:1020D000D578981893782D061B042B43157804396E
:1020E0002B43557804322D022B430360AFE7022ABD
:1020F0000AD1114AE05C511AE218527812020243E6
:102100000A6004339BB2B7E7012AB5D10A4A521AD2
:10211000E15C1160F5E7084959180A600433ACE73F
:10212000000004403C0004403800044034000440F7
:10213000300004400C00044000010440040004404E
:102140001000044014000440F7B5150080221C0064
:102150001023D2050091916807000B439360002380
:10216000654AD730136001F07FFD9D233E009B0040
:10217000F9583B00CA363200FC33002900D07FE01A
:10218000586801F001FE390032785C4BCB311A609F
:102190004B780A781B0213438A78AC4612041A4320
:1021A000CB78281D1B061343554A1BBA13604B7985
:1021B0000A791B0213438A7912041A43CB791B064E
:1021C0001343504A1BBA13604B7A0A7A1B0213431B
:1021D0008A7A12041A43CB7A21001B0613434A4A17
:1021E0001BBA1360009A2B021343484A1360220063
:1021F000474B1B1B0093009BCE785B1801938B7899
:1022000036061B0433430E78043833434E780431CA
:1022100036023343019E33600328ECDC0321A80817
:10222000431C9B002940800003292BD13849E51825
:102230005E18A9786D78E35C09042D0229431943DF
:102240003160030008330021FF2B2DDD314B324973
:1022500019600F21314B1960012327490B60304B66
:1022600019680029FCD006211B680B40042B20D0E4
:1022700080220020D20593680A318B439360FEBD13
:1022800001217DE7022908D121495D18E11849782B
:10229000E35C090219432960D3E70129D3D11C4922
:1022A0005918E35C0B60CCE7194818180160043337
:1022B000CAE7002310490B606346002B0CDC3B008F
:1022C000FC335A68102101325A608022D20593688B
:1022D00001208B439360D2E7009B9B181B68190A6F
:1022E00013705170190C1B0ED37004235B42917054
:1022F0009C440432E0E7C046000004403C00044037
:102300003800044034000440300004400C00044015
:102310000001044004000440080F000010000440C5
:102320001400044070B5061E19D002225A4B9B7946
:102330009343012B13D1594B1A78FF2A0FD15A78A6
:10234000FF2A0CD19A78FF2A09D1DA78FF2A06D120
:102350001A79FF2A03D15B79FF2B00D199E0504B0A
:102360000C201A78012A08D000224E4D1A702978C4
:102370000B00093B042B01D8212070BD4B1F012B02
:10238000FAD9454CA37B042B00D982E0A279032A19
:1023900000D97EE09A1ED2B2012A02D860881F2896
:1023A00077D9002E56D0012E73D1A0880128E3D012
:1023B000002907D1581E032803D801F0B7FB1217D4
:1023C00015122E702978481E032811D80025364B87
:1023D0001D602823237501F0A7FDA84227D0A58002
:1023E000CAE702212970EDE70421FBE70321F9E7A1
:1023F00007390129C0D82D490968C96A8906BBD5A2
:102400002B4908780028B7D1012A01D9002BB3D174
:1024100002230B708021274D2633890128782375EC
:1024200001F0A2FD80212878890101F0F5FC01234B
:10243000A380214B1B78002B0AD0FA2280211F4B4E
:1024400092001B8809025A431A4B187801F084FD48
:10245000002092E701F090FD2B78A680073B012B2E
:1024600003D917482E7001F0FFFC114B114C1A785C
:10247000002A06D080210022207889011A7001F0FC
:1024800073FD01F031FC80212078090201F06CFD20
:10249000DEE7122071E7C046A60BFF1F6B09FF1F86
:1024A0001A09FF1F1C09FF1F4809FF1F4464FF1F73
:1024B0002309FF1F1B09FF1F2109FF1F2C09FF1FF5
:1024C0000010004010B5002901D001F0F5FC10BD4E
:1024D000F7B5604B01919978A1239B004B435E4A6D
:1024E000060014681022E418D6235B00E058362357
:1024F000FF33E35C00279343222B41D1574B0F3A24
:102500001A600760012501F0FFFC019B1880E82399
:102510005B00E35C002B01D0B34258DD0023504F39
:10252000FB70AD33FF33E3581A68002A03D09B8851
:10253000DB439B071DD03823FF33E35C002B18D00F
:102540009B235B00E35C002B13D1D133FF33E35CAF
:10255000B3420EDAA4235B00E15AE018090A023103
:1025600001F0C2FC23000122FE33013E01351A872F
:10257000FA70E8235B00E35C002B2AD0A8B2FEBD12
:1025800003683D00002BBED081880430090A023167
:1025900001F0AAFCD6235B00E3581F60B2E72300DA
:1025A000B133BA00FF339858013781880430090AE3
:1025B000023101F099FCE8235B00E35CBB42EEDCF6
:1025C000E822F61AED1800235200A354A6E70027CC
:1025D000F1E7200001F030FB00281FD0002E1DDDA8
:1025E0007319882647190193B600200001F0FCFA00
:1025F0005A30800020184068013581880430090A6B
:10260000023101F071FC200001F0A6FBA359013357
:10261000A351BD4202D0019B9D42E6D1114BE35C28
:10262000002BABD095239B00E35C002BA6D00E4B78
:10263000E15A0029A2D00D4AA35C994202D9013384
:10264000A3549BE700231A212000A35401F0ACFB04
:1026500094E7C046300DFF1F3409FF1F00140340EC
:10266000E010FF1F5A020000720200005E0200002C
:102670000D4970B54A6E0D4CD2038B69D20BA24244
:1026800006D80B4D0224AA4204D901F0E5FA70BD28
:1026900002246442E21815007E2425402242F4D030
:1026A000A3432B438B61F0E700F000400A200000B9
:1026B000FC1C0000F8B51D4B1D4F1A78002A10D1E4
:1026C000BA7B002A02D101321A7003E0032AFAD041
:1026D000022AF8D001F028FC00220120154B1A70C4
:1026E000F8BD154B154D1C68154B9E7801232B70BA
:1026F0002878C0B200F0A2FBBB7B002B0BD101F00D
:102700005BFAA1239B007343E41883239B00E41826
:1027100023782B70E4E7032B02D101F09DFBF0E757
:102720000020022BDCD101F02FFCEAE71C09FF1F7F
:10273000A60BFF1F2309FF1F3409FF1F490AFF1FB4
:10274000300DFF1FF0B587B00EAD2F780FAD2D788F
:102750000593AC46634614000E4D0CAA12782E78F1
:1027600003930D9B009201932200059B029701F0B9
:102770004BFC2E70012C01D0042C08D1802206497C
:102780008B889343054A1278D20113438B8007B09C
:10279000F0BDC0461C09FF1F6C11FF1F7809FF1F09
:1027A0000B001B3B70B504003020E02B0DD813004C
:1027B000E025493BFF3B9BB2ED00AB4205D8034B04
:1027C000200019825A8201F057FA70BD8410FF1F51
:1027D00010B501F011FB054B00205B68052B04D9F7
:1027E000034A5268D20200D4980810BD001000407D
:1027F000FCE100E070B501F0BFFB0D4B1B68FC3342
:10280000DC691D6AFFF7E4FF6419844204D2094BB6
:1028100001241B68002B07D004220024064B1A70E9
:10282000064A93690133936101F05EFA200070BD9E
:102830004464FF1F9809FF1F2309FF1FFC0FFF1FA0
:1028400070B50C4D2B68FC335C6A01F095FBFFF70B
:10285000BFFF2B680025FC339B6AE318834204D238
:10286000054B1B68AB4200D1051B01F03DFA280067
:1028700070BDC0464464FF1F9809FF1FD722044B58
:1028800092009B5810B5002B00D0984710BDC04651
:102890000000FF1F10B501F0D3F8FFF7EFFF274945
:1028A000274BCA6D274C1A4084235B001343CB652A
:1028B000254B1B68186A01F0DFFA244B244A1A6082
:1028C000244B254A1A60A022244B52001A60244B44
:1028D000187801F051FA2000224901F09DFB0023F5
:1028E000A3600233A360204B2049236003232048C8
:1028F000A36001F091FB10221E4BFF201A60802282
:1029000052031A60802292031A60802212041A6015
:1029100001F01AFB012001F03FFAFA20400001F01B
:1029200063FA582001F058F9134801F045FA0120E4
:1029300001F072F9072001F04FFA10BD00F00040DD
:1029400000FEFEFF141000404464FF1F000003401F
:102950000180063DBC00034034080000A400034091
:102960004A0AFF1F71020000C3090000FFFF3F0079
:102970002810004000E100E030750000674E336829
:1029800088331B6883F3088801F0E6F8644A6549D8
:10299000136800200B401360634B644A1B6893422A
:1029A00000D1A6E001F070FA0221614A13688B435E
:1029B0001360FFF76FFF5F4B5F4C1878C0B201F0F8
:1029C00073FA0023A3600233A3605C4B01202360F1
:1029D00001F052FA0323A36001F016FA040001F09B
:1029E0000BFA050001F010FA554B186001F0E4FAFB
:1029F000544B1968621A531EA14200D21300802260
:102A0000D203934201D39B029B0A3268D16AC90761
:102A100000D471E04C491C0C09689BB24C435943EB
:102A20002402090A641803264849FC3293680A689C
:102A300047489B1A474A0768126847499B18474A04
:102A40009A1833409208DB190A600360042B03D9FB
:102A5000013233400A6003600E684149A619300014
:102A600001F08AF83F4F3E493B68C3183B60300095
:102A7000019301F011F93C4E306808183849306074
:102A8000884205D9019B01333B6001F005F93160B3
:102A900001F00AF9354B1B78002B0DD001F0ACF991
:102AA000334B621B196812188A4232D24919091B2A
:102AB000091A304801F0B0FA2F4E337A002B0ED0AD
:102AC00001F09AF9621BF1681218914224D9491950
:102AD000091B091A294801F09FFA00233372284B79
:102AE00083F3088801F090F8002001F0CDF901F09F
:102AF000ABFA01F0C9F95CE7DC0199000234641A11
:102B00005900641A09214B438033CB40A408E418D0
:102B100089E7FA218900CCE71A49DBE74464FF1F03
:102B20001CF00040FFFFC1FF0C0AFF1FB64121034C
:102B300010000040490AFF1F14100040C3090000A4
:102B4000100AFF1F340AFF1F380AFF1F200AFF1F49
:102B5000280AFF1F1C0AFF1F240AFF1FC4090000C8
:102B6000710200006008FF1F2C0AFF1F1C09FF1FD5
:102B7000E408FF1F00100040740BFF1F3C100040D2
:102B800000000020DC050000A022054B92009B58AD
:102B900010B5002B01D0984710BD01F045F8FBE7B8
:102BA0000000FF1FA122054B92009B5810B5002B7F
:102BB00001D0984710BD01F037F8FBE70000FF1F78
:102BC000A222054B92009B5810B5002B01D09847CC
:102BD00010BD01F029F8FBE70000FF1FA322054B01
:102BE00092009B5810B5002B01D0984710BD01F002
:102BF0001BF8FBE70000FF1FA422054B92009B5827
:102C000010B5002B01D0984710BD01F00DF8FBE77F
:102C10000000FF1F70B501F0EFF84F4B186001F096
:102C2000E3F90400C30702D401F06EF870BD00227E
:102C30004A4B1A604A4B18780138042829D800F00A
:102C400075FF0320181C2400200001F0ADF90128B5
:102C5000ECD0444C2378042B6ED100F095FF002873
:102C6000E4D001F0E1F9582000F0B6FF0223237010
:102C7000DCE7200001F008F8E9E7200001F0ACF9FA
:102C8000E5E7200001F038F8E1E7200000F09CFFC4
:102C9000DDE701F041F90500012808D1324B1B782E
:102CA000053B012B03D82000FFF76EFFD1E72D4B2A
:102CB0001B78022B01D0052B20D1022D28D12B4BC4
:102CC0009B7BAB431CD12000FFF76CFF264B187891
:102CD0000128BED16405BCD4244925224B7B034284
:102CE00005D1233A13405A42534126331A000B7D33
:102CF0009342AED9322000F0EFFFAAE7022D07D1B0
:102D0000194B1B78052B11D12000FFF759FFDDE788
:102D1000012D0BD1012B03D12000FFF75FFF98E7B6
:102D2000062B03D12000FFF767FF92E7200000F099
:102D30007BFF022D8DD1C9E7032B04D10C4B987C6E
:102D400000F0BAFF72E7072B00D06FE7094B987BC2
:102D500000F0F2FF6AE7C0469C09FF1F9809FF1FB9
:102D60009009FF1F2309FF1F1C09FF1FA60BFF1F50
:102D7000BC0BFF1FD40BFF1FFA210A4B0A4A490064
:102D80001A640A4A5A500A4A04395A50094A083100
:102D90009A64094A5A50094A5C315A50084ADA661C
:102DA0007047C0460000FF1F4527FF1F4128FF1F37
:102DB000F527FF1F2523FF1FB526FF1FC51DFF1F7A
:102DC000991DFF1F10B500F099FE10BDF7B50B0C53
:102DD000FF270122009300233C001E001D009446A3
:102DE000019089B262469A40100008401841361896
:102DF000B6B2FF2F02D1012E00D19FB2009802403F
:102E00001A41AD18ADB2FF2C02D1012D00D19CB2F8
:102E10000133102BE6D10320012E07D1012D04D15F
:102E2000019B2401E4191C700138FEBD102EFCD159
:102E30000238102DF9D00230F7E700008023F7B5F3
:102E40009C46264B264F01932649274A274D284C5E
:102E5000284B02281AD1604638600868264E304058
:102E6000802636033043086001990978002909D18A
:102E70001660224A2A60224A2260E02219689143A1
:102E8000A03A1BE08021C9021160F2E766463E606D
:102E90000F68194E3E408027FF023E430E600199A5
:102EA000097800290DD1176001280ED1154A2A6032
:102EB000154A2260E02219689143C03A0A431A6019
:102EC000F7BD802189021160EEE7E0210F4A02433D
:102ED0002A600F4A22601A688A43F0E74B0AFF1FF4
:102EE000E0000340D800034090000340000003408E
:102EF0005000034040000340FFFFE3FF0280063D17
:102F0000804508220180063D8066082200800698E0
:102F100080550822F8B51E4B80261A680020140040
:102F20003440324232D11A681A4F32431A600122B9
:102F30003B68063093433B6000F09EFF0122164D34
:102F40002B681E432E603B680A2613433B60802794
:102F5000BF00124B1B683B4211D1013EF6B2FF2E5F
:102F600009D17E220E4B1C682B68E40B144093435E
:102F700023432B6005E0082000F07EFFE9E7002EE8
:102F8000EFD180222B68600893432B60F8BDC046C8
:102F9000C4F000405CF0004018F0004068F00040D1
:102FA00060F0004010B500F027FE01215820034AD0
:102FB00000F0DAFDFFF7AEFF10BDC046600AFF1F4C
:102FC00010B578220021034800F07EFE01F014F8CD
:102FD000002010BD4C67FF1F70B5040000F0CCFF4F
:102FE00000230C200B4A010059438D18515C002925
:102FF0000DD0A14208D1012300246B7000F064FFC2
:1030000000F072FE200070BD01330A2BEBD11224B8
:10301000F6E7C0464C67FF1F70B5040000F0ACFF38
:10302000002319001D000D4A1078002806D0A04288
:103030000CD1557001310C320A29F5D1002B0AD17F
:1030400000F0DAFF00F050FE002070BD5078461E00
:10305000B0411B18EEE700F037FFF3E74C67FF1FA6
:10306000F7B504000C20002384460E4D01926746FC
:103070005F43E85D7E19A04212D000280BD10A4BB5
:103080009C4662461B7808331370019B70707C5518
:103090007160B360FEBD01330A2BE8D10320F9E76C
:1030A0000720F7E74C67FF1F4867FF1F8020F8B530
:1030B000484BC0051B68C1248360474BFF251A6835
:1030C000012313434361454BA4001A68444B40213C
:1030D0001A60444B1A68444B1A60444B1A59AA436D
:1030E0001A51C52292009E58AE4331438026995012
:1030F0009F583F49F6010F403E439E509E588027FF
:103100003602360A3043985080201A5900020A408D
:1031100002431A5104341A59364E3F043240802675
:103120003A431A511A5936061202120A32431A51F8
:1031300008341A5980260A4002431A51C3229200C9
:103140009F58B446AF4337439F509F58294E0F4076
:1031500007439F509F5837408026360437438026C8
:103160009F509F5836063F023F0A37439F50C02268
:103170001F59AF433A431A511A591202120A164301
:10318000C6221E5192009C58AC4365462C439C506D
:103190009C5800250C4020439850C72080001A58A6
:1031A000154C1140C02212020A431A50134B1B78CF
:1031B000DB08AB4201DC0020F8BD2378002B06D0F1
:1031C000A368002B00D0984701350C34EEE712209D
:1031D000F2E7C0466843FF1F6443FF1FB0F00040A2
:1031E0004467FF1FB4F000404067FF1F00E100E0AC
:1031F000FF00FFFFFFFF00FF4C67FF1F4867FF1F37
:10320000030010B51F2809D8072200201340072407
:1032100004490A78A24313430B7010BD0023062013
:10322000F5E7C0464867FF1F054B06491B780A684B
:1032300005485B0702401B0B134300200B607047DF
:103240004867FF1F1CF00040FFFFC1FF70B50C2551
:10325000FFF7EAFF0A4B1C780A4BE4086543ED18B8
:10326000002C01D1200070BD2B78002B06D06B689C
:10327000002B00D09847013C0C3DF1E71220F2E70B
:103280004867FF1F4067FF1F1FB5002102220B0088
:1032900001910091052000F0CFFE02230B490A683E
:1032A0001A42FCD120230393039B5A1E0392002B46
:1032B000FAD1074A1368002BFCDA0B246C44200077
:1032C000012100F0B9FD207804B010BD90C8004085
:1032D00000C8004013B504000A4B0193019B002B6A
:1032E00001D1112016BDFFF7CFFF23000340044298
:1032F00005D0052000F0C0FD019B013BEDE7180063
:10330000F0E7C046FFFFFF0707B500F035FE80225B
:103310000821D205936A0191002B01D107399162EE
:1033200002210C4A11600199481E01900029FAD12E
:1033300003311160053101910199481E0190002966
:10334000FAD11160002B02D18022D205936200F0E5
:10335000CBFC07BD00C00040F0B52D4C89B02378F0
:10336000002B4FD1FEF7CEFA02232A4F03903A6882
:103370001A42FCD120230693069B5A1E0692002B6C
:10338000FAD1254E3368002BFCDA0120FFF7A2FFAB
:10339000011E02D0112009B0F0BD030003220190EC
:1033A000009005AD9F2000F047FE0321280000F0AB
:1033B00043FD02233A681A42FCD120230793079B5E
:1033C0005A1E0792002BFAD13368002BFCDA012039
:1033D000FFF780FF0028DDD10398FEF7A7FAAA784F
:1033E0006B7811041B020B4329780B4363601300B5
:1033F000113B0A49052B07D801239340A3600B60BA
:10340000012323700020C6E780231B03F6E7C04694
:103410005043FF1F90C8004000C800409808FF1F9D
:103420001E4B30B55A6818781D4B85B0D3185942D9
:103430004B4101210093002300F0C6FD194B1A4AAD
:1034400002259A6300221A6510325A658022C4212F
:103450009D65164B1648D202DA6789004258154B13
:1034600080241A4080231B041343435064234120CB
:103470000393E40500F006FA402000F003FA6562C9
:10348000039D6B1E0393002DFAD103236362FFF7A4
:103490003BFFA562FFF760FF05B030BD5C43FF1F37
:1034A00095FFFEF700C80040050001FF04E100E0C1
:1034B00000E100E0FFFF00FFF0B585B00700FEF778
:1034C00021FA022305002D4C22681A42FCD1202348
:1034D0000093009B5A1E0092002BFAD1284E3368AD
:1034E000002BFCDA0120FFF7F5FE002803D01124A1
:1034F000200005B0F0BD234B2360022322681A424E
:10350000FCD120230193019B5A1E0192002BFAD17A
:103510003368002BFCDA0120FFF7DCFE0028E6D13F
:10352000194B1F60022322681A42FCD12023029308
:10353000029B5A1E0292002BFAD13368002BFCDA50
:103540000120FFF7C7FE0028D1D1104B23600223D2
:1035500022681A42FCD120230393039B5A1E039234
:10356000002BFAD13368002BFCDA0120FFF7B2FE02
:10357000041EBCD12800FEF7D9F9B9E790C8004075
:1035800000C8004001000006A8C8004001800001FA
:1035900010B50020FFF790FF10BD000010B5064BDE
:1035A00018705960FFF73CFF00211320034AFFF712
:1035B00057FD002010BDC0465C43FF1F2134FF1F94
:1035C000F0B5040085B003920291FEF79BF98822C2
:1035D00063035B0B52051A438023DB059D6A80233E
:1035E000274F0092BA68002601901B039A420CD91B
:1035F000F82326001B041E401C4206D08022214BCB
:1036000052025E6219680A431A60002D0BD100F065
:10361000B3FC02221C4B1A608023DB055A62013A7C
:103620009A6200F061FB0023039A934220D1002D9F
:103630000AD100F0A1FC144B03221D608023DB059E
:103640005A629D6200F050FB8023BA681B039A42C5
:1036500008D9002E06D000220A4B0C495A621A687B
:103660000A401A600198FEF761F9002005B0F0BD2C
:10367000009A0299D2181278CA540133D4E7C0468E
:103680005043FF1F00C8004000C00040FFFFFEFF86
:10369000F0B587B0029103920400FEF733F9019070
:1036A00000F06AFC802302250122234EDB053560F1
:1036B0005D629A6200F018FB204F3B682B42FCD100
:1036C00020230493049B5A1E0492002BFAD11C4D14
:1036D0002B68002BFCDA0120FFF7FCFD002802D04C
:1036E000112007B0F0BD2000039A029900F0D4FB2E
:1036F000022304003A681A42FCD120230593059B5B
:103700005A1E0592002BFAD12B68002BFCDA0120FF
:10371000FFF7E0FD051EE3D100F02EFC802303221D
:10372000DB0535605A629D6200F0DEFA0198FEF713
:10373000FDF8E0B2D5E7C04600C0004090C80040A8
:1037400000C80040F0B5802489B00600FEF7DAF822
:10375000E405A36A02250393029000F00DFC012307
:10376000304F3D606562A36200F0BEFA2E4C2368C4
:103770002B42FCD120230593059B5A1E0592002B5A
:10378000FAD12A4D2B68002BFCDA0120FFF7A2FDAD
:10379000002803D01124200009B0F0BD244B236081
:1037A000022322681A42FCD120230693069B5A1E4C
:1037B0000692002BFAD12B68002BFCDA0120FFF7D0
:1037C00089FD021EE6D11B4B03211E600300019000
:1037D0000090202000F030FC022322681A42FCD125
:1037E00020230793079B5A1E0792002BFAD12B68C0
:1037F000002BFCDA0320FFF76DFD041ECAD100F098
:10380000BBFB80230322DB053C605A629C6200F014
:103810006BFA039B002B01D1FFF776FD0298FEF7B0
:1038200085F8B8E700C0004090C8004000C80040DC
:103830000100000694C8004007B50002019104226F
:10384000000A01A9FFF724FF0EBD000073B50500B3
:1038500005240B4AA3005B429B1819686B46DE1DCA
:103860003000FFF7B3FA022804D133782B55013C1E
:10387000EFD276BD052CFCD00128FAD10230F8E752
:10388000140900111F2807D8012380228340D20584
:1038900091680B43936070473F2808D8012380222A
:1038A00020388340D20551690B435361F3E75F2809
:1038B000F1D80123802240388340D205116A0B439E
:1038C0001362E8E71F2807D8012280218240C9053A
:1038D0008B6893438B6070473F2808D80122802172
:1038E00020388240C9054B6993434B61F3E75F2859
:1038F000F1D80122802140388240C9050B6A9343E8
:103900000B62E8E71F2810D880230200DB05153A78
:103910001968012A06D820229143196019680A43C0
:103920001A60704701228240F6E73F2811D88023B1
:103930000200DB05353AD968032A06D810229143E4
:10394000D960D9680A43DA60EBE701222038824067
:10395000F5E75F28E5D842238022181A413B8340CF
:10396000D205516A99435162516A0B435362D8E7B9
:1039700010B50400012813D1A022184992050B6844
:103980005B015B0913430B60154B164A1968114024
:10399000154A0A431A60402219680A431A6010BD8A
:1039A0000028FCD101000A2000F056FB21000B206A
:1039B00000F052FBC0220A4B920019680A434021D2
:1039C0001A601A688A431A60B022044912060B680A
:1039D0005B015B0913430B60E1E7C04614F0004054
:1039E0001CF000407F00FEFF80FD010072B6074A18
:1039F0001368013313600422054B1A600023054A43
:103A000013608022D2055360FEE7C0467808FF1F8E
:103A1000C0F00040C4F0004005490B68002B05D100
:103A2000044A0A6004490A60044A13607047C046A9
:103A3000140AFF1F841E0000380AFF1FC4F0004054
:103A40000023034A1360034A1360034A136070475C
:103A500054F0004040F1004044F10040002310B514
:103A6000184C8AB0009301932378012B27D0694624
:103A7000012000F0D9F9002817D1009B12490293C8
:103A8000019B06AA0393114B02A81B680493104BD9
:103A90001B68059300F088F810220E4906A800F074
:103AA0001BFA002804D1FF23237000200AB010BDA8
:103AB0000123094A074902A8237000F075F8012084
:103AC000F4E7C0464864FF1F1029001108290011BF
:103AD0000C290011202900114C64FF1F13B501248B
:103AE0006946012000F0A0F9034B00940193FFF711
:103AF000B5FF200016BDC046BB0B000010B5FFF798
:103B00009FFFFFF7EBFF002802D0024B984710BD44
:103B1000FEE7C046E1A2000002B471464908490030
:103B2000095649008E4402BC7047C04602B4714633
:103B300049084900095C49008E4402BC7047C046F0
:103B400003B47146490840004900095A49008E44AF
:103B500003BC70470000000001B40248844601BC69
:103B6000604700BFC9A9000001B40248844601BCF7
:103B7000604700BF0167010001B40248844601BCF0
:103B8000604700BF090E000001B40248844601BC32
:103B9000604700BF01D7000001B40248844601BC61
:103BA000604700BFBD5C010001B40248844601BC0F
:103BB000604700BFDD3F000001B40248844601BCFD
:103BC000604700BFE9F6000001B40248844601BC2A
:103BD000604700BFF935010001B40248844601BCCA
:103BE000604700BF7912010001B40248844601BC5D
:103BF000604700BFD9B0000001B40248844601BC50
:103C0000604700BFED68010001B40248844601BC72
:103C1000604700BF7997000001B40248844601BCA8
:103C2000604700BFE512010001B40248844601BCB0
:103C3000604700BFE917010001B40248844601BC97
:103C4000604700BF71B0000001B40248844601BC67
:103C5000604700BFE90B010001B40248844601BC83
:103C6000604700BFD1AE000001B40248844601BCE9
:103C7000604700BF8944000001B40248844601BC8B
:103C8000604700BF116E000001B40248844601BCC9
:103C9000604700BF0934010001B40248844601BCFA
:103CA000604700BF090E000001B40248844601BC11
:103CB000604700BFD544010001B40248844601BCFE
:103CC000604700BF4DF9000001B40248844601BCC2
:103CD000604700BFB70E000001B40248844601BC33
:103CE000604700BF6137010001B40248844601BC4F
:103CF000604700BF9DA9000001B40248844601BC92
:103D0000604700BFF535010001B40248844601BC9C
:103D1000604700BFDD0A010001B40248844601BCCF
:103D2000604700BF51B8000001B40248844601BC9E
:103D3000604700BFEDB5001101B40248844601BCE4
:103D4000604700BFC1F7000001B40248844601BCCF
:103D5000604700BFE94C010001B40248844601BC41
:103D6000604700BF5976010001B40248844601BC97
:103D7000604700BFE927000001B40248844601BC47
:103D8000604700BFEDA5000001B40248844601BCB5
:103D9000604700BF2144000001B40248844601BCD2
:103DA000604700BF6911010001B40248844601BCAC
:103DB000604700BF53B9000001B40248844601BC0B
:103DC000604700BF8D11010001B40248844601BC68
:103DD000604700BF8937010001B40248844601BC36
:103DE000604700BFF90D010001B40248844601BCE0
:103DF000604700BF8512010001B40248844601BC3F
:103E0000604700BFC95C010001B40248844601BCA0
:103E1000604700BF156B010001B40248844601BC35
:103E2000604700BF0D52010001B40248844601BC46
:103E3000604700BFE1AC000001B40248844601BC09
:103E4000604700BF3D71010001B40248844601BCD7
:103E5000604700BFF9ED000001B40248844601BC90
:103E6000604700BF75F8000001B40248844601BCF9
:103E7000604700BFC1A5000001B40248844601BCF0
:103E8000604700BF0189000001B40248844601BCBC
:103E9000604700BF016C010001B40248844601BCC8
:103EA000604700BF9573010001B40248844601BC1D
:103EB000604700BF8914010001B40248844601BC78
:103EC000604700BFE9D4000001B40248844601BC49
:103ED000604700BF21A9000001B40248844601BC2C
:103EE000604700BFCD4C010001B40248844601BCCC
:103EF000604700BFC115010001B40248844601BCFF
:103F0000604700BF8D82000001B40248844601BCB6
:103F1000604700BFCD0C010001B40248844601BCDB
:103F2000604700BFDD0C010001B40248844601BCBB
:103F3000604700BFA9D8000001B40248844601BC14
:103F4000604700BF85C1000001B40248844601BC3F
:103F5000604700BFED6B010001B40248844601BC1C
:103F6000604700BF8B52010001B40248844601BC87
:103F7000604700BFB352010001B40248844601BC4F
:103F8000604700BF75A9000001B40248844601BC27
:103F9000604700BF19FA000001B40248844601BC22
:103FA000604700BF6D0B010001B40248844601BCAC
:103FB000604700BF0134010001B40248844601BCDF
:103FC000604700BFC166010001B40248844601BCDD
:103FD000604700BFC56D010001B40248844601BCC2
:103FE000604700BF0534010001B40248844601BCAB
:103FF000604700BFBD0B010001B40248844601BC0C
:10400000604700BFADAE000001B40248844601BC69
:10401000604700BF9D6A000001B40248844601BCAD
:10402000604700BF2D6C010001B40248844601BC0A
:10403000604700BF6DF6000001B40248844601BC31
:10404000604700BF496D010001B40248844601BCCD
:10405000604700BF8552010001B40248844601BC9C
:08406000604700BF69A20011D6
:1040680002000000C2BE001101000000B0BC001137
:1040780002000000BEBE001101000000A840FF1FA2
:1040880002000000B8BC001101000000C061FF1F61
:1040980002000000BCBE0011030000003461FF1FD5
:1040A8001200000002000000C2BE00110100000062
:1040B800F8BC001102000000BEBE001101000000A3
:1040C800F5BC00110200000002BD00110300000051
:1040D8006F61FF1F02000000BCBE0011030000005A
:1040E8008461FF1F02000000BEBE00110100000035
:1040F800F4BC00110200000000BD00110300000024
:104108004561FF1F02000000BCBE00110300000053
:104118006661FF1F02000000C2BE0011010000001E
:104128003CBD001102000000BEBE001101000000ED
:10413800F141FF1F020000004EBD00110100000008
:1041480033BD001102000000BEBE001101000000D6
:10415800F041FF1F020000004CBD001101000000EB
:104168008C61FF1F02000000BEBE001101000000AC
:10417800EF41FF1F020000004ABD001101000000CE
:1041880023BD001102000000BEBE001101000000A6
:10419800EE41FF1F0200000048BD001101000000B1
:1041A8001EBD001102000000BEBE0011010000008B
:1041B800ED41FF1F0200000046BD00110100000094
:1041C80019BD001102000000BEBE00110100000070
:1041D800EC41FF1F0200000044BD00110100000077
:1041E80014BD0011020202020202000000000000D9
:1041F80014130000A94B00116F4B001190BD001162
:1042080090011D0018001800FFFF070102030405B4
:104218000602010600000000000000000000000087
:104228000000000000000000000000000000000086
:104238000300000002000000C2BE001101000000DF
:10424800B0BD001102000000BEBE00110100000058
:10425800AC42FF1F02000000BABD001101000000BF
:10426800BA61FF1F02000000BCBE0011030000007D
:104278002464FF1F02000000BEBE00110100000000
:10428800AC42FF1F02000000B8BD00110100000091
:10429800BC61FF1F02000000BCBE0011030000004B
:1042A8001C64FF1F12006C6C00000000000000007E
:1042B80000000000080700000001000000000111D4
:1042C800FFFF0000504859360000000000000000C1
:1042D8000B000500F0000000B400002800280028AA
:1042E8003075A000A000A000A00000080008E001B0
:1042F800F000100010001000100010001000500016
:104308005000500010001000D0070000000000000E
:104318000F0001000500307507001000010081FF43
:1043280000000000FF0000005174001159720011D4
:10433800E96F0011FFFF0100FF0000006D9E0011F2
:10434800E99B0011019B0011000000000000000023
:1043580000000800040000003B0001085902E001C9
:1043680088212800FF00000002000000C2BE0011E2
:104378000100000088BF001102000000BEBE00114D
:1043880001000000ED43FF1F02000000BABE00114B
:10439800010000000468FF1F02000000BEBE0011FB
:1043A80001000000EC43FF1F02000000B8BE00112E
:1043B80001000000EA43FF1F02000000BEBE00111A
:1043C80001000000E843FF1F02000000B6BE001114
:1043D80001000000E043FF1F180018001D009001B5
:1043E800020000030202000002000000C2BE001129
:1043F800010000009CBF001102000000BEBE0011B9
:10440800010000003044FF1F02000000B4BE00118C
:10441800000000000000000002000000BCBE001107
:0A442800030000002468FF1F20FFBE
:040000051FFF184180
:00000001FF
